:10142400758400852ED2852FD37584018530D285AD
:1014340031D3E4F52FF52E30005730064E855B820C
:10144400855A83E0F52FA3E0F52EA385825B85837F
:101454005AE55B655D700CE55A655C7006755B006A
:10146400755A02855982855883E533F0A3E532F035
:10147400A3858259858358E559655D7014E55865DF
:101484005C700E755900755802800685322E8533BE
:101494002F30010CE52E2534F52EE52F3535F52FAB
:1014A400300210E53F8527F0A4252EF52EE5F03512
:1014B4002FF52F300310E50A852AF0A4252EF52EEA
:1014C400E5F0352FF52F300410E5118529F0A4251A
:1014D4002EF52EE5F0352FF52FE4F531F5303009F2
:1014E4005730054E855B82855A83E0F531A3E0F5DC
:1014F40030A385825B85835AE55B655D700CE55A94
:10150400655C7006755B00755A028559828558833F
:10151400E535F0A3E534F0A3858259858358E55970
:10152400655D7014E558655C700E75590075580258
:10153400800685343085353130080CE5302532F5A8
:1015440030E5313533F531300A10E53F8527F0A415
:101554002530F530E5F03531F531E531C3952C40D2
:0315640003852CD0
:1015670031300B10E50A852AF0A42530F530E5F077
:101577003531F531300C10E5118529F0A42530F50A
:1015870030E5F03531F531300D10E5188528F0A438
:101597002530F530E5F03531F531E531C3952D408E
:1015A70003852D31229016053015031215C230160A
:1015B700031215D23018031215F522E50B2509F58C
:1015C7000BE50C3508F50C93F50A22E512250EF507
:1015D70012E513350DF51393C313F8E5142510F52C
:1015E70014E515350FF51593C31328F51122E519E1
:1015F7002517F519E51A3516F51A93F518227F827E
:1016070085888C8F9295989B9EA1A4A7AAADB0B30D
:10161700B6B9BBBEC1C3C6C9CBCED0D3D5D7D9DC2B
:10162700DEE0E2E4E6E7E9EBEDEEF0F1F2F4F5F601
:10163700F7F8F9FAFBFCFCFDFDFEFEFEFEFEFEFEE2
:10164700FEFEFEFDFDFCFCFBFAFAF9F8F7F6F4F3F3
:10165700F2F0EFEDECEAE8E7E5E3E1DFDDDBD8D632
:10166700D4D1CFCDCAC8C5C2C0BDBAB7B4B2AFAC6A
:10167700A9A6A3A09D9A9794908D8A8784817E7A44
:101687007774716E6B6865625F5C595653504D4A4B
:101697004744423F3C393734322F2D2A282624210C
:1016A7001F1D1B1918161412110F0E0C0B0A080711
:1016B7000605040403020201010000000000000007
:1016C70000000001010202030405060708090A0BCE
:1016D7000D0E1011131516181A1C1E202224272967
:1016E7002B2E303335383A3D404245484B4E515406
:1016F70056595C606366696C6F7275787B7FFEFE16
:10170700FEFEFDFCFCFBFAF8F7F6F4F3F1EFEDEB68
:10171700E9E7E4E2DFDCDAD7D4D0CDCAC6C3BFBC81
:10172700B8B4B0ACA8A39F9B96928D89847F7A7535
:10173700706B66615C57514C47413C37312C262111
:101747001B16100B050000050B10161C21272C3249
:10175700373D42484D53585D62686D72777C81858D
:101767008A8F94989DA1A5AAAEB2B6BABEC1C5C8C4
:10177700CCCFD2D5D8DBDEE1E3E6E8EBEDEFF1F253
:10178700F4F6F7F8F9FBFBFCFDFEFEFEFEFE000C8F
:101797001926333F4C5864707B86919CA6AFB8C11D
:1017A700C9D1D8DEE4EAEFF3F6F9FCFDFEFEFEFD53
:1017B700FCFAF7F4F0EBE6E0DAD4CCC5BCB4ABA1A5
:0E17C700978D83786D61554A3D3125180C00D1
:101E6000D2F4C2F5C2F675840F85F0C812254A7403
:101E700003121EAF12253E7403121EAF122521124B
:101E800025217403121EAF1225217402121EAF12F7
:101E900025217428121F1B7406121F1B740E121F9B
:101EA0001B7401121F1B12253E7480121F1B22C0BF
:101EB00000A2E092F3A2E192F2A2E292F1A2E392F6
:101EC000F0D2F475840F85F0C8C2F47830D8FE855E
:101ED000F0C87830D8FED00022C00075840FA2E48C
:101EE00092F3A2E592F2A2E692F1A2E792F0D2F486
:101EF00085F0C8C2F47830D8FE85F0C87830D8FEB6
:101F0000D00022EF75840FD2F5C2F685F0C8121EFC
:101F1000D9122521121EAF1225212275840FC2F578
:101F2000C2F685F0C8121ED9122521121EAF122545
:101F30002122EF14A2E492E6C2E4D2E7121F1B2290
:101F4000740F121F1B22740D121F1B227F01121F00
:101F50003278107F20121F03D8F9227F11121F320E
:101F600078107F20121F03D8F9227F01121F3278C8
:101F7000207F20121F03D8F922C0077F018004C0F0
:101F8000077F11121F32D007C082C083C007EF75D0
:101F9000F010901FAA1225627810E493FF121F031D
:091FA000A3D8F7D007D083D0824A
:101FA9002220202020202020202020202020202026
:101FB9002057414954494E4720464F522052494ED5
:101FC900472054454C434F20414E535745524544B1
:101FD90020205741495420464F5220444953434FEA
:101FE9002020205445535420204641494C45442043
:101FF9002020205445535420205041535345442018
:10200900202020454550524F4D20544553542020FF
:1020190020204155582052454C415920544553548C
:102029002020205055534820544F2054414C4B20D8
:102039002054455354203320434841522F5355428D
:102049002054455354204649584544205354524935
:102059004E544553542056415249422053545249F3
:102069004E464143544F52592044454641554C54DC
:102079002050524F4752414D4D494E47204D4F44F4
:102089004553494D504C45582052455045415445BA
:10209900522020205245434F5244494E4720202088
:0120A9002016
:102AC60032C28D32758400C2CF32C0E0C083C0826C
:102AD600C0D0C000C0F0C2CFB21A201A23121424EC
:102AE600151BE51B7009751B0A7584017588AF15E2
:102AF6001CE51C7009751C607584027588AF801111
:102B06001215AC1536E5367008753604758400D294
:102B16008B758400D2ECD0F0D000D0D0D082D08398
:102B2600D0E032C2CF32C0E0C0D0C007C000C08300
:102B3600C08212443275888FD082D083D000D007ED
:102B4600D0D0D0E032C0E0C0D0C000C083C082C0C8
:102B56008420121375840F30DF27E5E8540FF54003
:102B6600D2127541C8801A1541E5417006E540D27A
:102B7600E7F54075840F20DF08C212D211D22AD29F
:102B86002D20141475840F30F828E5E854F0C4F5A8
:102B960042D2147543C8801A1543E5437006E542D0
:102BA600D2E7F54275840F20F808C214D213D22951
:102BB600D21C124477151DE51D702A751D0A124494
:102BC6009E151EE51E701E751E0A1244F1151FE5A0
:102BD6001F7012751F061244F21526E5267006753B
:102BE600260A1244FBD084C28DD082D083D000D076
:102BF600D0D0E0323220100DD21085BF3585BE34DC
:0A2C060075BB01800BC21085BF33BF
:102C100085BE3275BB00C2ED32C0E0C0D0E544B421
:102C2000000A054485BE3F75BB07803DB4010A0517
:102C30004485BE3C75BB048030B4020A054485BEA1
:102C40003F75BB068023B4030A054485BE3D75BBB2
:102C5000048016B4040A054485BE3F75BB0580098F
:102C600075440085BE3E75BB04C2EDD0D0D0E032C5
:103E590044313233343536373839302A23414243F5
:103E6900202020205354414E444259202020202014
:103E7900524144494F204F524947494E41544520E8
:103E890054454C434F204F524947494E41544520D0
:103E990020202046554E4354494F4E2031202020A2
:103EA90020202046554E4354494F4E203220202091
:103EB90020202046554E4354494F4E203320202080
:103EC90020202046554E4354494F4E20342020206F
:103ED90020202046554E4354494F4E20352020205E
:103EE90020202046554E4354494F4E20362020204D
:103EF90020202046554E4354494F4E20372020203C
:103F090020202046554E4354494F4E20382020202A
:103F190020202046554E4354494F4E203920202019
:103F2900202052454345495645204D4F44452020C0
:103F3900205452414E534D4954204D4F4445202061
:103F4900202045204C4541442044454C41592020DE
:103F5900205741495420464F52204D204C45414459
:104504001268C8124A8475840F1200A41268BC127F
:1045140061DA1262131264D712598A20A503120EAB
:10452400DA9000A5E4F020A432302915C229E5422E
:10453400540FFFEF903E5993FF90008CEFF0125010
:1045440068302AE2C22AE540540FFFEF903E5993A7
:10455400FF90008BEFF012514B80CB9000A5E0FF51
:10456400EF124235458D00459201459702459C0363
:1045740045A10445A60545AC0645B20745B808451E
:10458400BE0945C40A0000452A125D1180981246EE
:104594008E8093125794808E1265048089122C7039
:1045A4008084122FB102452A1250DA02452A126081
:1045B4007902452A125BEE02452A1266CF02452A89
:0A45C400124C2102452A02452A226A
:105D11001266B51268B01268BC1267AE12644C12FA
:105D210064D7125DE412697E9000ACE4F09000B19A
:105D3100E4F09000A6E4F09000EEE4F09000EDE4D1
:105D4100F07BFF7A3E79691263C0121F5B753832AE
:075D51009000A5E004F02220
:10468E00E538600302474C124B9F125508302B0B36
:10469E001265A7C22B9000A5E4F022301F0B126208
:1046AE004CC21F9000A5E4F02212676650409000A5
:1046BE00E1E0FF9000A7EFF09000EBE0FFEFB40217
:1046CE00031268AA9000ECE0FFEFB402031268B682
:1046DE009000B1E4F07BFF7A3E79891263C07BFFD4
:1046EE007A3F79491263F19000A57402F0221267A5
:1046FE0078EF604A9000EAE0FFEF60421267BE90EA
:10470E0000E2E0FF9000A8EFF09000EBE0FFEFB4C6
:10471E0002031268AA9000ECE0FFEFB402031268E5
:10472E00B69000B1E4F07BFF7A3E79791263C07BDC
:0F473E00FF7A3F79591263F19000A57406F022BB
:10579400121B759000A7E0FFEF702D1267BE9000FA
:1057A400EBE0FFEFB402031268AA9000ECE0FFEF15
:1057B400B402031268B675370A7BFF7A3F7929125F
:1057C40063F19000A57403F0124B9F302B0B12650C
:1057D400A7C22B9000A5E4F022301F0A12624CC22B
:0757E4001F9000A5E4F02274
:10650400121B75E53770231269661269331266B57A
:106514009000D8E0FF9000A3EFF09000EDE4F0903D
:0B65240000EEE4F09000A57405F022EA
:102C700020A6031253D8126930121B751217D512F1
:102C80005299125508123F69124B9F9000EEE0FFD7
:102C9000EF603F1266B51267AE9000EBE0FFEF64A5
:102CA0000160099000EBE0FFEFB402031268B090FE
:102CB00000ECE0FFEF640160099000ECE0FFEFB48E
:102CC00002031268BC9000EF740AF09000A574092A
:102CD000F0229000DBE0FFEF705C9000A6E0FFEFD9
:102CE000602B900098E0FFEF70239000A6E4F09036
:102CF0000099E4F09000DEE0FF9000D9E0FEEE2FB6
:102D0000FF9000A1EFF09000A5740AF022900098C7
:102D1000E0FFEF702190009CE0FFEF70199000DE63
:102D2000E0FF9000D9E0FEEE2FFF9000A1EFF090C1
:102D300000A5740AF0229000DBE0FFEFB4012190BF
:102D40000098E0FFEF70199000DEE0FF9000D9E0FE
:102D5000FEEE2FFF9000A1EFF09000A5740AF02284
:102D60009000DBE0FFEFB4022190009CE0FFEF70E9
:102D7000199000DEE0FF9000D9E0FEEE2FFF9000FA
:102D8000A1EFF09000A5740AF0229000DBE0FFEFC5
:102D9000D3940240219000B1E0FFEF70199000DE63
:102DA000E0FF9000D9E0FEEE2FFF9000A1EFF09041
:102DB00000A5740AF022302B201266B51268B012FA
:102DC00068BC1267AE1265A7C22B1269511269570F
:102DD0001269339000A5E4F022301F1D1266B5126F
:102DE00068B01268BC1269511269571269331262D5
:102DF0004CC21F9000A5E4F02212676640189000B4
:102E0000DEE0FF9000D9E0FEEE2FFF9000A1EFF092
:072E10009000A57408F022F8
:102FB10020A6031253D81267ED1265F5121B751284
:102FC10017D5126957126951125299125508123FB9
:102FD10069124B9F9000EEE0FFEF603F1266B51261
:102FE10067AE9000EBE0FFEF640160099000EBE059
:102FF100FFEFB402031268B09000ECE0FFEF640150
:1030010060099000ECE0FFEFB402031268BC90008D
:10301100EF740AF09000A57409F0229000DBE0FF44
:10302100EF701A900098E0FFEF700E90009CE0FFA7
:10303100EF600A126778EF7004125D9F229000DB47
:10304100E0FFEFB4010C900098E0FFEF6004125D27
:103051009F229000DBE0FFEFB4021290009CE0FFA2
:10306100EF600A126778EF7004125D9F229000DB17
:10307100E0FFEFB4030C9000B1E0FFEF6004125DDC
:103081009F229000DBE0FFEFB4040C9000B1E0FF61
:10309100EF6004125D9F22302B201266B51268B0DA
:1030A1001268BC1267AE1269691265A712695112E2
:1030B1006969C22B9000A5E4F022301F1D1266B58C
:1030C1001268B01268BC126951126933126969122F
:1030D100624CC21F9000A5E4F022126766404012C4
:1030E10067AE1266B59000EBE0FFEF6401600990F6
:1030F10000EBE0FFEFB402031268B09000ECE0FFD8
:10310100EF640160099000ECE0FFEFB40203126884
:10311100BC1269511269571269339000A5E4F0227B
:1050DA00125508126778EF600A9000E2E0FF90002C
:1050EA00A8EFF09000A8E0FFEF70299000E2E0FF3F
:1050FA00EF60211267AE9000EBE0FFEFB4020312FB
:10510A0068B09000ECE0FFEFB402031268BC9000B4
:10511A00A5E4F022126766500975370A9000A57453
:10512A0007F0124B9F302B0B1265A7C22B9000A5DC
:10513A00E4F022301F0A12624CC21F9000A5E4F06C
:01514A002242
:10607900126766400375370AE537701275370A7B70
:10608900FF7A3F79291263F19000A57403F0124B4E
:106099009F302B0B1265A7C22B9000A5E4F022308C
:0D60A9001F0A12624CC21F9000A5E4F022F5
:105BEE009000A1E0FFEF70401267AE1266B5900014
:105BFE00EBE0FFEF640160099000EBE0FFEFB40211
:105C0E00031268B09000ECE0FFEF640160099000B1
:105C1E00ECE0FFEFB402031268BC1269511269572F
:095C2E001269339000A5E4F02294
:1066CF009000EFE0FFEF700E1269511269571269D7
:0766DF00339000A5E4F02256
:104C21009000A1E0FFEF7004126389221269301233
:104C31001B751217D5123F69124B9F302B0B126552
:104C4100A7C22B9000A5E4F022301F0B12624CC2C8
:104C51001F9000A5E4F0229000EEE0FFEF603E120D
:104C610066B51267AE9000EBE0FFEF64016009905A
:104C710000EBE0FFEFB402031268B09000ECE0FF3C
:104C8100EF640160099000ECE0FFEFB402031268E9
:0E4C9100BC9000EF740AF09000A57409F022A8
:105D9F00126969126981125D581269339000E8E047
:105DAF00FFEF60069000AE7401F012669B9000EB5F
:105DBF00E0FFEFB401031268AA9000ECE0FFEFB42C
:105DCF0001031268B67BFF7A3F79391263F19000B5
:055DDF00A57404F02290
:106389007BFF7A3F79291263F11269331269661228
:1063990066B59000EBE0FFEFB401031268B090001E
:1063A900ECE0FFEFB401031268BC9000A57405F09E
:0163B90022C1
:1067AE009000E0E0FFEF60041268C2221268C82277
:1067BE009000E0E0FFEF60041268C8221268C22267
:106766009000DFE0FFEF60061268F2B322221268A3
:02677600F2220D
:10406A00900091E0FF703B9000CAE060159000CB91
:10407A00E0FEE53ED39E40249000CCE090009302FF
:10408A0041229000CBE0FEE53EC39E500F9000CC4B
:10409A00E0900093F09000917403F022E490009471
:1040AA00F022EF640170249000CBE024FBFFE53E90
:1040BA00D39F406C900093E06003024165900094A6
:1040CA0004F09000CDE0900092804D900091E0FFC6
:1040DA00B402179000CBE024FBFEE53ED39E4002DB
:1040EA00805F900092E070738066EF640370339093
:1040FA0000CBE02405FFE433FEC3E53E9FEE648077
:10410A00F8748098501A900093E0704F90009404CD
:10411A00F09000CDE0900092F0900091E004F0223F
:10412A008034900091E06404702C9000CBE0240568
:10413A00FFE433FEC3E53E9FEE6480F87480985036
:10414A00099000CDE0900092F022900092E0700B6E
:0C415A00900094F08001E4900091F022AD
:1054A700900091E0700E1268CE50559000CCE090BD
:1054B7000093801E900091E0B401221268CE501A2A
:1054C700900093E0701790009404F09000CDE09066
:1054D7000092F0900091E004F022E4801F90009188
:1054E700E0B4021C1268CE50099000CDE090009203
:1054F700F022900092E07008900094F0900091F0F4
:015507002281
:0D67ED009000C9E060030254A712406A2228
:103F6900900095E0FF703B9000CEE060159000CF87
:103F7900E0FEE53DD39E40249000D0E090009702FA
:103F890040299000CFE0FEE53DC39E500F9000D040
:103F9900E0900097F09000957403F022E490009867
:103FA900F022EF640170259000CFE024FBFFE53D8E
:103FB900D39F4074900097E0701290009804F0909D
:103FC90000A6F09000D1E09000968054900095E012
:103FD900B402179000CFE024FBFFE53DD39F4002D8
:103FE9008064900096E07002806B900095E0FF6419
:103FF9000370379000CFE02405FDE433FCE53DC3B1
:104009009DEC6480F8748098501E900097E0701AB7
:1040190090009804F09000A6F09000D1E0900096EE
:10402900F0900095E004F0228031EF6404702C9048
:1040390000CFE02405FFE433FEC3E53D9FEE648035
:10404900F874809850099000D1E0900096F0229081
:104059000096E07006900098F08001E4900095F0D9
:014069002234
:10529900900099E070191268DA500E9000D4E090ED
:1052A900009BF0900099E004F0E490009CF02290BB
:1052B9000099E0B401221268DA501A90009BE0705C
:1052C9001790009C04F09000D5E090009AF09000AF
:1052D90099E004F022E4801F900099E0B4021C12C6
:1052E90068DA50099000D5E090009AF02290009A6F
:0C52F900E0700890009CF0900099F022FA
:1055080090009DE0700E1268D450559000D2E09043
:10551800009F801E90009DE0B401221268D4501AAA
:1055280090009FE070179000A004F09000D3E090E6
:10553800009EF090009DE004F022E4801F90009D02
:10554800E0B4021C1268D450099000D3E090009E89
:10555800F02290009EE070089000A0F090009DF06E
:015568002220
:106778009000D7E060069000A0E0FF22900094E02F
:02678800FF22EE
:1065F5009000D8E0FF601D90009CE070069000A020
:10660500E060069000A3EFF0229000A3E0700590F3
:05661500009004F022DA
:104FF50054564F582020434F53202053454E534578
:10500500004F4E202020202020202020202020205E
:1050150020004F4646202020202020202020202030
:10502500202000191823A01296203D129623A012C5
:105035009627631488203D148823A01488276316B7
:10504500B8203D16B823A016B827631918203D19B6
:1050550018276312962B8C14882B8C16B82B8C1959
:03506500182B8C79
:104A840012690C1269091268CEE433F54F12690FEA
:104A9400E433F54F126912E433F54F126915E43328
:104AA400F54F126918E433F54F12691BE433F54FDF
:104AB40012691EE433F54F126921E433F54F12698C
:104AC40024E433F54F1268E0E433F54F126927E428
:104AD40033F54F1268ECE433F54F12692A12692D4D
:104AE40012693612693912693C12693F126942121D
:104AF400694512694812694B12695A12695D126953
:104B04006012696312696C12696F126972126975B5
:064B140012697802697BC2
:0668AA0075840FD2FC22F0
:0668B00075840FC2FC22FA
:0668B60075840FD2B72229
:0668BC0075840FC2B72233
:0668C20075840FD2FE22D6
:0668C80075840FC2FE22E0
:10669B0075840FD2FD9000EBE0B401031268AA9051
:0A66AB0000ECE0B401031268B6220F
:1066B50075840FC2FD9000EBE0B401031268B09041
:0A66C50000ECE0B401031268BC22EF
:03690900C2932214
:03690C00D2932201
:0668CE0075840FA2FA22FE
:03690F00A2A02221
:03691200A2A1221D
:03691500A2A22219
:03691800A2A32215
:03691B00A2A42211
:03691E00A2A5220D
:03692100A2A62209
:03692400A2A72205
:0668D40075840FA2F922F9
:0668DA0075840FA2DD220F
:0668E00075840FA2DE2208
:03692700A2922217
:0668E60075840FA2DA2206
:0668EC0075840FA2DB22FF
:0668F20075840FA2DC22F8
:0668F80075840FA2D822F6
:0668FE0075840FA2D922EF
:03692A00D208226E
:03692D00C208227B
:03693000D2092267
:03693300C2092274
:03693600D20A2260
:03693900C20A226D
:03693C00D2022262
:03693F00C202226F
:03694200D20B2253
:03694500C20B2260
:03694800D20C224C
:03694B00C20C2259
:03694E00D20D2245
:03695100C20D2252
:03695400D2182234
:03695700C2182241
:03695A00D20E2238
:03695D00C20E2245
:03696000D20F2231
:03696300C20F223E
:03696600D200223A
:03696900C2002247
:03696C00D2012233
:03696F00C2012240
:03697200D203222B
:03697500C2032238
:03697800D2042224
:03697B00C2042231
:105D5800E4FDFCED25E0FFEC33FE74002FF58274C2
:105D6800023EF583E4F0A3F00DBD00010CBC0EE388
:105D7800BDE0E07558027559007402F55AF55B905C
:105D880000D9E075F0BEA4AEF02400F55DEE340253
:065D9800F55CC200D2051B
:015D9E0022E2
:03697E00C205222D
:105DE400E4FDFCED25E0FFEC33FE74002FF5827436
:105DF400023EF583E4F0A3F00DBD00010CBC0EE3FC
:105E0400BDE0E07558027559007402F55AF55B90CF
:105E140000D9E075F0BEA4AEF02400F55DEE3402C6
:045E2400F55CD20651
:015E28002257
:03698100C2062229
:0B682A0075081575095ED215D2032217
:0B68350075081575095ED215D20B2204
:07689C00C215C203C20B226A
:0B6840009000BD12328CD216D2042250
:0B684B009000BE12328CD216D20C223C
:0C328C00E0F529E4F512F513F514F51532
:10329800EF12423533932333822A32D03032E2316F
:1032A80032F432330633331834332A35333C363369
:1032B8004E3733603833713933A44133B54233C69E
:1032C8004333D744000033EF905028E493F50D744E
:1032D8000193F50E90502A0233E690502CE493F5B2
:1032E8000D740193F50E90502E0233E6905030E4A1
:1032F80093F50D740193F50E9050320233E6905019
:1033080034E493F50D740193F50E9050360233E6CC
:10331800905038E493F50D740193F50E90503A02ED
:1033280033E690503CE493F50D740193F50E9050FC
:103338003E0233E6905040E493F50D740193F50E88
:103348009050420233E6905044E493F50D74019393
:10335800F50E9050460233E6905048E493F50D740C
:103368000193F50E90504A807590504CE493F50DFA
:10337800740193F50E90504E8064905050E493F58C
:103388000D740193F50E9050528053905054E4936D
:10339800F50D740193F50E9050568042905058E404
:1033A80093F50D740193F50E90505A803190505C4E
:1033B800E493F50D740193F50E90505E80209050C3
:1033C80060E493F50D740193F50E905062800F90B0
:1033D8005064E493F50D740193F50E905066E493F0
:0833E800F50F740193F51022AA
:0768A300C216C20CC2042260
:05690400C215C20322D0
:0B6856007508027509ABD215D20B22A9
:0B68610075081A7509ABD215D20B2286
:1053D8001252991255087BFF7A4F79F51263C090E3
:1053E800009CE07BFF60067A50790680047A507949
:1053F800171263F17F17121F32AF3E1225A79000D4
:105408006CE0FF121F0390006DE0FF121F03900075
:105418006EE0FF121F037F1C121F32AF3D1225A73B
:1054280090006CE0FF121F0390006DE0FF121F0355
:0854380090006EE0FF021F036B
:10024D0020202020202020202020202020202020A1
:10025D002020202020202020202020202020202091
:10026D002054454C434F2050524F4752414D202072
:10027D0020524144494F2050524F4752414D20206A
:10028D002054574F20544F4E45204D4F444520206C
:10029D0020434F4D50552050524F4752414D202035
:1002AD00202041434345535320434F4445202020B4
:1002BD0044544D462054454C434F204C4556454CD7
:1002CD0044544D4620524144494F204C4556454CCF
:1002DD004245455020524144494F204C4556454CCE
:1002ED00424545502054454C434F204C4556454CB6
:1002FD0054454C434F20524144494F204C45564C98
:10030D00524144494F2054454C434F204C45564C87
:10031D00524144494F204C494D4954204C45564C6F
:10032D002045494120544F4E45204C4556454C20C3
:10033D004C4F57204755415244204C4556454C2073
:10034D0048494748204755415244204C4556454C55
:10035D00564F494345205241444930204C45564C57
:10036D00564F4943452054454C434F204C45564C20
:10037D0020434F53204F5220535155454C43482055
:10038D002020434F5320504F4C4152495459202067
:10039D00434F53205452494747455220564F4C54D2
:1003AD00434F5320414351554953542054494D45D2
:1003BD00434F532052454C454153452054494D45DB
:1003CD002053454E534520504F4C415249545920CE
:1003DD0053454E205452494747455220564F4C5491
:1003ED0053454E20414351554953542054494D4591
:1003FD0053454E2052454C454153452054494D459A
:10040D005220564F582041435155495354494F4E50
:10041D0020525820564F582052454C4541534520A7
:10042D005420564F582041435155495354494F4E2E
:10043D0020545820564F582052454C454153452085
:10044D00204F5045524154494E47204D4F44452071
:10045D0020564F58204F5220434152524945522069
:10046D002020564F58204143544956495459202075
:10047D00202054454C434F2044454C4159202020C9
:10048D002020524144494F2044454C4159202020C1
:10049D0053454E53452C20564F582C20544F4E4506
:1004AD0020204143434553532044454C415920207E
:1004BD00205455524E204F4E2044454C415920203A
:1004CD00205455524E204F46462044454C4159200C
:1004DD004449474954414C20494E20504F4C4152BC
:1004ED00434E544C2052454C415920504F4C415293
:1004FD002020452D44454C41592050425820202064
:10050D002020452D44454C41592052454320202063
:10051D00202052494E474F5554204D4F44452020E1
:10052D00414E535745522052494E47204E4D42524F
:10053D0020202052494E4720535041434520202032
:10054D00202052494E4720414E53574552202020DE
:10055D0052494E47205452414E534954494F4E53E0
:10056D0045494120544F4E4520454E41424C452072
:10057D0046554E4354494F4E20382053454C454324
:10058D00524144494F2053454C454320454E424C22
:10059D00204155582052454C4159204D4F4445203E
:1005AD002043542052454C4159204D4F4445202065
:1005BD00202020202020202020202020202020202E
:1005CD00202020202020202020202020313D454E9D
:1005DD002020202020202020202020524154494F2F
:1005ED002020202020202020202020303D434F534C
:1005FD002020202020202020202020313D504F532E
:10060D0020202020202020202020202031204D536C
:10061D0020202020202020202020203130204D534C
:10062D0020202020202020202020313030204D532C
:10063D002020202020202020202020202053454332
:10064D00202020202020202020202020204D494E19
:10065D002020202020202020202020204D4F4445E8
:10066D002020202020202020202020313D564F58B2
:10067D00202020202020202020202052494E47538A
:10068D0020202020202020202020204359434C458D
:10069D0020202020202020202020313D544F4E4569
:1006AD002020202020202020504F4C4152495459C9
:1006BD008201001102381500018201011103381564
:1006CD000001820102110438150001820103110598
:1006DD003815000178060411060119000082030A7D
:1006ED001107391500FF82030B1108391500FF8220
:1006FD00030C1109391500FF82030D110A3915007C
:10070D00FF82030E110B391500FF82030F110C39F7
:10071D001500FF820310110D391500FF8203111111
:10072D000E391500FF820312110F391500FF8203D8
:10073D00131110391500FF8203141111391500FF23
:10074D008203151112391500FF82011611133A1586
:10075D00000182011711143B1500018203181115B8
:10076D00391500FF82021911163C15006382021A19
:10077D0011173D15006382011B11183B15000182F5
:10078D00031C1119391500FF82021D111A3C1500A9
:10079D006382021E111B3D15006382021F111C3C5A
:1007AD00150063820220111D3E1500638202211186
:1007BD001E3C150063820222111F3E15006382014B
:1007CD00231120411500028201241121421500013F
:1007DD0082022511224015006382022611233D1548
:1007ED00002882022711243D150028820128112599
:1007FD004115000482022911263E150A6382022A40
:10080D0011273C15006382022B11283D15006382D0
:10081D00012C11294615000182012D112A461500C2
:10082D000182022E112B3D1501FF82022F112C3E4C
:10083D00150063820130112D3C150001820131112B
:10084D002E43150009820232112F3C1500638201DF
:10085D00331130411500018203341131441501FF6C
:10086D0082013511323815000182013611334515DB
:10087D00000182013711343815000182013811351C
:10088D004115000382013911364115000320202046
:10089D002020202020202020202020202082010127
:1008AD0011020C15000120202020202020202020C6
:1008BD0020202020202082010111020C1500012092
:1008CD0020202020202020202020202020202064D7
:1008DD0001001102091500012020202020202020D8
:1008ED0020202020202020200101010101010101F3
:1008FD0001000000000000000000000000000000EA
:10090D0000000000000000000000000000000000DA
:10091D0000000000000000000000000000000000CA
:10092D0000000000000000000000000000000000BA
:10093D0000000000000000000000000000000000AA
:10094D0000002020202020202020202020202020DA
:10095D002020010101010101010101000000000041
:10096D00000000000000000000000000000000007A
:10097D00000000000000000000000000000000006A
:10098D00000000000000000000000000000000005A
:10099D00000000000000000000000000000000004A
:1009AD0000000000000000000000000020202020BA
:1009BD0020202020202020202020202001010101A6
:1009CD000101010101000000000000000000000015
:1009DD00000000000000000000000000000000000A
:1009ED0000000000000000000000000000000000FA
:1009FD0000000000000000000000000000000000EA
:100A0D0000000000000000000000000000000000D9
:100A1D000000000000002020202020202020202089
:100A2D0020202020202082010011021E150001012E
:100A3D00010101313233343536FF323232FFFFFFDF
:100A4D00550CFF3232000180000A0080000A000AB6
:100A5D00000A0001002828001E140000012863016F
:100A6D000163000A01010102000000000000000006
:100A7D0044313233343536373839302A2341424305
:100A8D0044AAA3C1C2C3C4D7ABA8A92A23414243D8
:100A9D0036333036373036393437313937343437F9
:100AAD0037303739373832353835343838353931DC
:100ABD0035393438393734313030313033313037EE
:100ACD0031313031313431313831323331323731F6
:100ADD0033313133363134313134363135313135DD
:100AED0036313539313632313635313637313731B8
:100AFD0031373331373731373931383331383631A2
:100B0D003839313932313936313939323033323091
:100B1D003632313032313832323532323932333396
:100B2D003234313235303235343030363030373092
:100B3D003135303137303231303233303235303289
:100B4D00363033313033323033363034333034376E
:100B5D003035303035313035333035343036353061
:100B6D00373130373230373330373431313431314A
:100B7D003531313631323231323531333131333243
:100B8D00313334313431313433313435313532312F
:100B9D00353531353631363231363531373231370B
:100BAD003432303532313232313432323332323511
:100BBD0032323632343332343432343532343632F2
:100BCD0035313235323235353236313236333236E1
:100BDD0035323636323731323734333036333131D0
:100BED0033313533323533333133333233343333C9
:100BFD0034363335313335363336343336353337A2
:100C0D0031343131343132343133343233343331B0
:100C1D003433323434353434363435323435343487
:100C2D00353534363234363434363534363635306F
:100C3D00333530363531363532333532363533326C
:100C4D003534363536353630363631323632343651
:100C5D003237363331363332363534363632363640
:100C6D00343730333731323732333733313733323C
:100C7D0037333437343337353441424344454647AF
:100C8D0048494A4B4C4D4E4F50515253545556575F
:100C9D0058595A6162636465666768696A6B6C6D01
:100CAD006E6F707172737475767778797A303132C0
:100CBD0033343536373839607E21402324255E267E
:100CCD002A28295F2D2B3D7B7D5B5D7C3A3B3C3E8D
:100CDD002C2E3F2F202020202020202020202020BF
:100CED0020474C4F42414C202020202020204354AF
:100CFD0043535320434F444520202020202020449F
:100D0D00435320434F44452020202020204C545253
:100D1D0020524550454154455220202020535045E6
:100D2D004544204449414C494E47202020535045CD
:100D3D0045442043414C4C494E47202020205054DF
:100D4D0043204E554D424552202020202020564F05
:100D5D00494345204D455353414745532020564F58
:100D6D0049434520504C41594241434B2020204995
:100D7D004E56414C49442054595045202020204F77
:100D8D005554204F462052414E4745202020494C76
:100D9D004C4547414C2056414C554520204D55530F
:100DAD00542046494C4C204649454C44202020496E
:100DBD004C4C4547414C20434F4445202020444155
:100DCD00544120414343455054454420204C494E05
:100DDD0045204E554D4245523A2020202055534531
:100DED00522050524F4752414D4D494E4755534554
:100DFD00522049443A2020202020202020564F49BF
:100E0D004345205245434F5244494E472020494CBB
:100E1D004C4547414C20454E545259202020494CB9
:100E2D004C4547414C2047414E4720202020202053
:100E3D00434F4D504C455445442020202020474CD5
:100E4D004F42414C20454550524F4D2020202043CC
:100E5D005443535320454550524F4D2020202020C0
:100E6D0044435320454550524F4D202020202020F3
:100E7D004C545220454550524F4D2020202044497E
:100E8D00414C494E4720454550524F4D202043413E
:100E9D004C4C494E4720454550524F4D2020202067
:100EAD0050544320454550524F4D2020202052454F
:100EBD0050454154455220454550524F4D202049F3
:0D0ECD004E495449414C495A494E47202096
:10624C009000A47464F0E4900000F030200B301F38
:10625C0024125F3812271A80F530210B301F1612CA
:10626C005F7A12271A80F530220B301F081229137F
:06627C0012271A80F52232
:10271A009000A4E07012900000E0D394004009C237
:10272A0020C221C222C21F22900000E01242352894
:10273A003300283601283902283C03283F0428415F
:10274A0005284306284507284808284B0A284E0B1F
:10275A0028510F285410285714285A15285D19286B
:10276A00601A28631B28661E28691F286C23286F95
:10277A002428722828752928782D287B2E287E2F30
:10278A00288130288432288733288934288C3528B0
:10279A008F64289265289566289867289B6E289DDD
:1027AA006F289F7028E17128A17828A37928A57A33
:1027BA0028E17B28A78228A98328AB8428AD85280D
:1027CA00B08C28B38D28B58E28B78F28BA9628BD25
:1027DA009728BF9828C19928C4A028C7A128CAA2A7
:1027EA0028CCA328CFAA28D1AB28D4AC28D6AD2888
:1027FA00D9B428DCB528DFB628E1B728E3BE28E635
:10280A00BF28E9C028ECC128E1C228F2F028F5F176
:10281A0028F8F228FBFA28FEFB2901FC2904FD29E5
:10282A0007FE290AFF0000290D02678A02665E0276
:10283A005E29026559800480028000025BA402318D
:10284A00210263220233F002584102353E025895B2
:10285A0002368C025FBC0255C9023BC4025A2902E5
:10286A0037DA025A75023928025AC1023A760264E4
:10287A007B0261A1025C37125B590256E0800002BA
:10288A00522B025EF50258E9025E6D02628202571D
:10289A003A80468032804B80408022804580078083
:1028AA0026803F025B0D0245CE801C803502593AD4
:1028BA00024C9F8008802B025FFB0247FF0251BC3B
:1028CA00802002474D8012024E928016023D0F026E
:1028DA004E1602536F800B800C024F0B0259DA021C
:1028EA00494F0260B60257EB026580025305026740
:1028FA00CE02568402698D02698E02698F024D1CCE
:09290A00026990E4900000F02243
:10678A00E4900002F09000A47464F0900000E00429
:02679A00F022EB
:10665E00121F4C121F5B7BFF7A0D79EA1263C07F0B
:0F666E0011121F32C226C223900000E004F02256
:105E2900302340900001E0FFC223BF2A0790000001
:105E3900E004F022EF6423702A7F23121F039000ED
:105E490002E004F0E0C394034013C220C221C2223D
:105E5900C21FE4900000F012652F021F6A90000033
:035E69007402F0D0
:015E6C002213
:106559007BFF7A0D79EA1263C0121F5B7F11121F4C
:10656900321267FAE490003CF07F2A121F03C22618
:07657900900000E004F02295
:105BA400302346900001E0F55EC223E55E642A607E
:105BB40038AF5E1267DE5022AF5E121F0390003CC6
:105BC400E02403F582E43400F583E55EF090003CC4
:105BD400E004F0900000E004F0227BFF7A0E791AD2
:095BE4001263C090000074FAF095
:015BED002295
:1031210020230302328B900001E0FFC223BF2A0754
:103131009000007403F022EF6423600302327C12DA
:103141001F03900004E064397077A3E06439707163
:10315100A3E06439706BD227900003E0FFB431081B
:10316100E4900036F00231EBEFB43208E49000371E
:10317100F00231FEEFB43302803E900003E0FFB471
:103181003408E4900038F002322CEFB43508E490B2
:103191000039F0023242EFB43608E490003AF0020E
:1031A1003258EFB437028010900003E0B438028047
:1031B10007900003E0B4390B7BFF7A0E792A0232C3
:1031C10082C227900003E0FFB43016A3E0B43011AF
:1031D100A3E0B4300CA3E0B43007900000740AF00F
:1031E10022EFB4310C1256275007900000740FF0F3
:1031F10022900003E0B4320C125569500790000090
:103201007414F022900003E0B43311A3E0B4300C45
:1032110012663D50079000007419F022900003E0FF
:10322100B4340FA3E0B4300A1266FD900000741E9E
:10323100F022900003E0B4350FA3E0B4300A126726
:10324100129000007423F022900003E0B4360FA323
:10325100E0B4300A1267279000007428F022900031
:1032610003E0B43716A3E0B43011A3E0B4300CA3EB
:10327100E0B43007900000742DF0227BFF7A0E79C4
:0A3281001A1263C090000074FAF006
:01328B002220
:1063220090003B740BF090003C7407F0E49000493D
:10633200F090004A743AF0E490004BF07BFF7A0C44
:1063420079EA1263C01263EB7F1E121F32900000C3
:046352007432F0228F
:1033F000124F80D3900072E09434900071E09400FA
:10340000400A1263BA90000074FAF022900071E052
:10341000FEA3E0FF9006BD75F009124229EE75F09B
:1034200009A42583F583E493900040F09006BE75CF
:10343000F009EF124229EE75F009A42583F583E423
:1034400093900041F0900071A3E09006BF75F009E1
:10345000124229EE75F009A42583F583E4939000C8
:1034600042F09006C075F009EF124229EE75F0099E
:10347000A42583F583E493900043F0900071A3E0CA
:103480009006C175F009124229EE75F009A4258352
:10349000F583E493FD900044F09006C275F009EFC7
:1034A000124229EE75F009A42583F583E493900078
:1034B00045F0900071A3E09006C375F0091242290F
:1034C000EE75F009A42583F583E493900046F0900F
:1034D00006C475F009EF124229EE75F009A42583A0
:1034E000F583E493900047F0900071A3E09006C547
:1034F00075F009124229EE75F009A42583F583E4DD
:1035000093900048F0ED6015900044E075F010A431
:10351000244DF9740235F0FA7BFF1263C090004528
:10352000E0FF601175F010A4244DF9740235F0FA33
:0E3530007BFF1263F1900040E0900000F0225B
:1058410090003B7410F090003C7407F09000497494
:105851003AF0E490004AF0900036E090004BF07B83
:10586100FF7A0C79FA1263C01263EB7F0D121F32BB
:10587100900004E0FF121F03900005E0FF121F03D8
:10588100900006E0FF121F037F1E121F32900000DE
:045891007432F0225B
:10353E00124F80D3900072E09400900071E09400DE
:10354E00400A1263BA90000074FAF022900071E003
:10355E00FEA3E0FF9008AA75F009124229EE75F05D
:10356E0009A42583F583E493900040F09008AB7591
:10357E00F009EF124229EE75F009A42583F583E4D4
:10358E0093900041F0900071A3E09008AC75F009A3
:10359E00124229EE75F009A42583F583E493900079
:1035AE0042F09008AD75F009EF124229EE75F00960
:1035BE00A42583F583E493900043F0900071A3E07B
:1035CE009008AE75F009124229EE75F009A4258314
:1035DE00F583E493FD900044F09008AF75F009EF89
:1035EE00124229EE75F009A42583F583E493900029
:1035FE0045F0900071A3E09008B075F009124229D1
:10360E00EE75F009A42583F583E493900046F090BF
:10361E0008B175F009EF124229EE75F009A4258361
:10362E00F583E493900047F0900071A3E09008B208
:10363E0075F009124229EE75F009A42583F583E48D
:10364E0093900048F0ED6015900044E075F010A4E2
:10365E00249AF9740835F0FA7BFF1263C090004586
:10366E00E0FF601175F010A4249AF9740835F0FA91
:0E367E007BFF1263F1900040E0900000F0220C
:1058950090003B7415F090003C7407F0900049743B
:1058A5003AF0E490004AF0900037E090004BF07B2E
:1058B500FF7A0D790A1263C01263EB7F0C121F3257
:1058C500900004E0FF121F03900005E0FF121F0384
:1058D500900006E0FF121F037F1E121F329000008A
:0458E5007432F02207
:10368C00124F80D3900072E09400900071E094008F
:10369C00400A1263BA90000074FAF022900071E0B4
:1036AC00FEA3E0FF9008C375F009124229EE75F0F5
:1036BC0009A42583F583E493900040F09008C47529
:1036CC00F009EF124229EE75F009A42583F583E485
:1036DC0093900041F0900071A3E09008C575F0093B
:1036EC00124229EE75F009A42583F583E49390002A
:1036FC0042F09008C675F009EF124229EE75F009F8
:10370C00A42583F583E493900043F0900071A3E02B
:10371C009008C775F009124229EE75F009A42583AB
:10372C00F583E493FD900044F09008C875F009EF20
:10373C00124229EE75F009A42583F583E4939000D9
:10374C0045F0900071A3E09008C975F00912422968
:10375C00EE75F009A42583F583E493900046F09070
:10376C0008CA75F009EF124229EE75F009A42583F9
:10377C00F583E493900047F0900071A3E09008CBA0
:10378C0075F009124229EE75F009A42583F583E43E
:10379C0093900048F0ED6015900044E075F010A493
:1037AC0024B3F9740835F0FA7BFF1263C09000451E
:1037BC00E0FF601175F010A424B3F9740835F0FA29
:0E37CC007BFF1263F1900040E0900000F022BD
:105FBC007BFF7A0D791A1263C07BFF7A0D79FA1286
:105FCC0063F17F0E121F32900005E0FF121F039049
:105FDC000006E0FF121F037F1A121F3290003B7461
:0F5FEC001AF090003C7404F09000007432F02220
:1055C9003028079000007403F0221263EB7F1E124B
:1055D9001F32125440900073E0FEA3E0FFD3940001
:1055E900EE9400402FEF94FBEE9400502790003B7F
:1055F900741BF090003C7407F0900049743AF0E491
:1056090090004AF0900035E01490004BF0900000B3
:0E5619007432F0221263BA90000074FAF0228C
:103BC400D3900072E09400900071E09400400A12D7
:103BD40063BA90000074FAF022900071E0FEA3E052
:103BE400FF9008DC75F009124229EE75F009A4254E
:103BF40083F583E493900040F09008DD75F009EFBD
:103C0400124229EE75F009A42583F583E49390000C
:103C140041F0900071A3E09008DE75F0091242298A
:103C2400EE75F009A42583F583E493900042F090A7
:103C340008DF75F009EF124229EE75F009A4258317
:103C4400F583E493900043F0900071A3E09008E0C2
:103C540075F009124229EE75F009A42583F583E471
:103C640093FD900044F09008E175F009EF124229A9
:103C7400EE75F009A42583F583E493900045F09054
:103C84000071A3E09008E275F009124229EE75F084
:103C940009A42583F583E493900046F09008E37526
:103CA400F009EF124229EE75F009A42583F583E4A7
:103CB40093900047F0900071A3E09008E475F00938
:103CC400124229EE75F009A42583F583E49390004C
:103CD40048F0ED6015900044E075F010A424CCF990
:103CE400740835F0FA7BFF1263C0900045E0FF6072
:103CF4001175F010A424CCF9740835F0FA7BFF1286
:0B3D040063F1900040E0900000F0220E
:105A290090003B741FF090003C7407F0900049749B
:105A39003AF0E490004AF0900038E090004BF07B97
:105A4900FF7A0D792A1263C01263EB7F0F121F329E
:105A5900900005E0FF121F03900006E0FF121F03EC
:0C5A69007F1E121F329000007432F022E9
:1037DA00124F80D3900072E09400900071E0940040
:1037EA00400A1263BA90000074FAF022900071E065
:1037FA00FEA3E0FF9008F575F009124229EE75F074
:10380A0009A42583F583E493900040F09008F675A7
:10381A00F009EF124229EE75F009A42583F583E435
:10382A0093900041F0900071A3E09008F775F009B9
:10383A00124229EE75F009A42583F583E4939000DA
:10384A0042F09008F875F009EF124229EE75F00976
:10385A00A42583F583E493900043F0900071A3E0DC
:10386A009008F975F009124229EE75F009A425832A
:10387A00F583E493FD900044F09008FA75F009EF9F
:10388A00124229EE75F009A42583F583E49390008A
:10389A0045F0900071A3E09008FB75F009124229E7
:1038AA00EE75F009A42583F583E493900046F09021
:1038BA0008FC75F009EF124229EE75F009A4258378
:1038CA00F583E493900047F0900071A3E09008FD1F
:1038DA0075F009124229EE75F009A42583F583E4EF
:1038EA0093900048F0ED6015900044E075F010A444
:1038FA0024E5F9740835F0FA7BFF1263C09000459D
:10390A00E0FF601175F010A424E5F9740835F0FAA7
:0E391A007BFF1263F1900040E0900000F0226D
:105A750090003B7424F090003C7407F0900049744A
:105A85003AF0E490004AF0900039E090004BF07B4A
:105A9500FF7A0D793A1263C01263EB7F0F121F3242
:105AA500900005E0FF121F03900006E0FF121F03A0
:0C5AB5007F1E121F329000007432F0229D
:10392800124F80D3900072E09400900071E09400F0
:10393800400A1263BA90000074FAF022900071E015
:10394800FEA3E0FF90095F75F009124229EE75F0B9
:1039580009A42583F583E493900040F090096075ED
:10396800F009EF124229EE75F009A42583F583E4E6
:1039780093900041F0900071A3E090096175F009FF
:10398800124229EE75F009A42583F583E49390008B
:1039980042F090096275F009EF124229EE75F009BC
:1039A800A42583F583E493900043F0900071A3E08D
:1039B80090096375F009124229EE75F009A4258370
:1039C800F583E493FD900044F090096475F009EFE5
:1039D800124229EE75F009A42583F583E49390003B
:1039E80045F0900071A3E090096575F0091242292D
:1039F800EE75F009A42583F583E493900046F090D2
:103A0800096675F009EF124229EE75F009A42583BD
:103A1800F583E493900047F0900071A3E090096764
:103A280075F009124229EE75F009A42583F583E49F
:103A380093900048F0ED6015900044E075F010A4F4
:103A4800244FF9740935F0FA7BFF1263C0900045E2
:103A5800E0FF601175F010A4244FF9740935F0FAED
:0E3A68007BFF1263F1900040E0900000F0221E
:105AC10090003B7429F090003C7407F090004974F9
:105AD1003AF0E490004AF090003AE090004BF07BFD
:105AE100FF7A0D794A1263C01263EB7F0D121F32E8
:105AF100900005E0FF121F03900006E0FF121F0354
:0C5B01007F1E121F329000007432F02250
:103A7600124F80D3900072E09400900071E09400A1
:103A8600400A1263BA90000074FAF022900071E0C6
:103A9600FEA3E0FF9009C975F009124229EE75F000
:103AA60009A42583F583E493900040F09009CA7534
:103AB600F009EF124229EE75F009A42583F583E497
:103AC60093900041F0900071A3E09009CB75F00946
:103AD600124229EE75F009A42583F583E49390003C
:103AE60042F09009CC75F009EF124229EE75F00903
:103AF600A42583F583E493900043F0900071A3E03E
:103B06009009CD75F009124229EE75F009A42583B6
:103B1600F583E493FD900044F09009CE75F009EF2B
:103B2600124229EE75F009A42583F583E4939000EB
:103B360045F0900071A3E09009CF75F00912422973
:103B4600EE75F009A42583F583E493900046F09082
:103B560009D075F009EF124229EE75F009A4258304
:103B6600F583E493900047F0900071A3E09009D1AB
:103B760075F009124229EE75F009A42583F583E450
:103B860093900048F0ED6015900044E075F010A4A5
:103B960024B9F9740935F0FA7BFF1263C090004529
:103BA600E0FF601175F010A424B9F9740935F0FA34
:0E3BB6007BFF1263F1900040E0900000F022CF
:10647B003022079000007401F02290003B742EF044
:10648B0090003C7407F07BFF7A0D795A1263C012AF
:0E649B0063EB7F1E121F329000007432F0225D
:1061A100302807900000742FF02290000AE0643834
:1061B1006005A3E0B4390A1263BA90000074FAF0E2
:1061C100227BFF7A0E790A1263C090000AE0540F15
:0961D100F5489000007430F02242
:105C370090000AE064386005A3E0B4390A1263BA39
:105C470090000074FAF0227BFF7A0D796A1263C024
:105C570090000AE0540FF548D202D20A9000C8E03B
:105C6700F527122E177BFF7A0E793A1263C0C2020C
:095C7700C20A90000074FEF02244
:105B590090000AE0540FF548302002D200122E2995
:105B690030201B201304E53B70F9122E20C2007B64
:105B7900FF7A0E793A1263C090000074FEF030216A
:105B890019201104E53B70F9122E207BFF7A0E795A
:0B5B99003A1263C090000074FEF0227E
:1056E000302356900001E0FF900034F0C223121FD7
:1056F00003900034E0FF1267DE5021900034E0FF99
:1057000090003CE02403F582E43400F583EFF09050
:10571000003CE004F0900000E004F022900034E04F
:10572000B42A079000007403F0227BFF7A0E791AE6
:0A5730001263C090000074FAF0222A
:10522B0030236A900001E0FF900034F0C223121F7C
:10523B0003900034E0FFB42A0B90003BE090000099
:10524B00F0D22822EFB4230B90003BE0900000F04B
:10525B00C22822900034E0FF1267DE502190003408
:10526B00E0FF90003CE02403F582E43400F583EF8B
:10527B00F090003CE004F0900000E004F0227BFF93
:0E528B007A0E791A1263C090000074FAF022B5
:105EF50030233F900001E0FF900034F0121F03C2F1
:105F050023900034E0FFB42A0B90003BE0900000A2
:105F1500F0D22822EFB4230B90003BE0900000F074
:105F2500C228227BFF7A0E791A1263C09000007492
:035F3500FAF0225D
:0A58E900900043E0FF700330283800
:1058F300121F3212661A124A2D8F5E900041E05237
:105903005EE55E60047F3180027F30121F03302822
:1059130017C228E55E2430900023F0900033740111
:08592300F090000074F0F02286
:0F592B00900046E0FF121F32900000E004F022CF
:105E6D00302340900001E0FF900034F0C223121F58
:105E7D0003900034E0FFB42A079000007403F02271
:105E8D001267DE500F900034E090000DF09000008E
:105E9D00E004F0227BFF7A0E791A1263C0900000A5
:045EAD0074FAF02271
:10628200302332900001E0FF900034F0C223BF2A95
:10629200079000007403F022900034E0B4230790CA
:1062A2000000E004F0227BFF7A0E791A1263C0909C
:0662B200000074FAF02266
:10573A0012661A900075EEF0A3EFF0124A2D8F4F01
:10574A0090003D7401F090000DE0B43108900041E2
:10575A00E0424F800E90000DE0B4301E900041E010
:10576A00F4524F900075E0FEA3E0FFAD4F1249ECF2
:10577A0012673C90000074FEF0227BFF7A0E791AC1
:0A578A001263C090000074FAF022D0
:104F0B00900043E0FF7003302856121F3212661ACE
:104F1B00900075EEF0A3EFF0E4F54F900041E0FF49
:104F2B00E54FC39F5027900075E475F001124213B3
:104F3B00AFF0FE124A2D8F507423254FF582E434C7
:104F4B0000F583E550F0121F03054F80CE3028107B
:104F5B00C228E54F04900033F090000074F0F0226B
:104F6B0090003C740AF0900046E0FF121F32900054
:054F7B0000E004F0223B
:104E9200302375900001E0FF900034F0C223121F0E
:104EA20003900034E0FFB42A079000007403F0225C
:104EB200EFB42308900000E004F080391267DE505E
:104EC20038900034E0FF90003CE0FE04F074032EC2
:104ED200F582E43400F583EFF0900041E02409FF0D
:104EE200E433FE90003CE0D39FEE6480F874809837
:104EF2004016900000E004F0227BFF7A0E791A122D
:094F020063C090000074FAF02273
:1060B600302337900001E0FF900034F0C223121F16
:1060C60003900034E0FFB42A079000007403F02226
:1060D600EFB42307900000E004F0227BFF7A0E79EC
:0B60E6001A1263C090000074FAF02250
:1057EB0012661A900075EEF0A3EFF090003C740A6D
:1057FB00F0E4F54F900041E0FFE54FC39F50279039
:10580B000075E475F001124213AFF0FE90003CE01E
:10581B00FD04F074032DF582E43400F583E0FD12F2
:10582B0049EC054F80CE7BFF7A0E793A1263C0901C
:06583B00000074FEF022E3
:1051BC0030236B900001E0FF900034F0C223121FEB
:1051CC0003900034E0FFB42A079000007403F0222F
:1051DC001267DE501A900034E0FF90003CE0FE04B1
:1051EC00F074032EF582E43400F583EFF080107B2D
:1051FC00FF7A0E791A1263C090000074FAF02290B4
:10520C000041E02409FFE433FE90003CE0D39FEE24
:0F521C006480F87480984006900000E004F0224F
:1045CE00900043E0FF7006202803024679121F3246
:1045DE0012661A900075EEF0A3EFF0124A2D122516
:1045EE00A7900041E0B4011090006EE0FF121F038F
:1045FE0090006EE0900023F0900041E0B402209015
:10460E00006DE0FF121F0390006EE0FF121F03907B
:10461E00006DE0900023F090006EE0900024F0908A
:10462E000041E06403703090006CE0FF121F0390B5
:10463E00006DE0FF121F0390006EE0FF121F03904B
:10464E00006CE0900023F090006DE0900024F0905C
:10465E00006EE0900025F0302811C228900041E055
:10466E00900033F090000074F0F022900046E0FFCE
:10467E00121F3290003C740AF0900000E004F02209
:105B0D001225FD5002803B1225D58F4F900047E0A6
:105B1D00FFE54FC39F402B900048E0FFE54FD39F1B
:105B2D00502012661A900075EEF0A3EFF0AD4F12F3
:105B3D0049EC7BFF7A0E793A1263C090000074FE37
:0C5B4D00F0221263BA90000074FAF022FB
:10593A001225FD5002803F1225D58F4F900047E077
:10594A00FFE54FC39F400B900048E0FFE54FD39F10
:10595A004004E54F702012661A900075EEF0A3EF2E
:10596A00F0AD4F1249EC7BFF7A0E793A1263C09080
:10597A00000074FEF0221263BA90000074FAF0225A
:104C9F00900043E0FF700330285E121F3212661A35
:104CAF00900075EEF0A3EFF0124A2D8F4F124B1AB2
:104CBF00E4F54F746C254FF582E43400F583E0FF83
:104CCF007423254FF582E43400F583EFF0746C25DF
:104CDF004FF582E43400F583E0FF121F03054FE523
:104CEF004FC3940440CD30280FC228900033740373
:104CFF00F090000074F0F022900046E0FF121F3297
:0D4D0F0090003C740AF0900000E004F022D7
:105FFB007F0A12425B8F4FE54F601212661A9000B8
:10600B0075EEF0A3EFF0E54F14FD1249ECE54F7B75
:10601B00FF600E7A0E793A1263C090000074FEF0A6
:0F602B00227A0D79BA1263C090000074FAF02245
:1047FF00900043E0FF700620280302489A121F32F0
:10480F0012661A900075EEF0A3EFF0124A2D1225E2
:10481F00A7900075E475F001124213AFF0FE124A33
:10482F002D12258B90006DE0FF900023F0A3F01266
:10483F001F0390006EE0FF121F03900075E475F0E8
:10484F0001124213AFF0FE124A2D12258B90006C0D
:10485F00E0FF900025F090006DE0900026F09000B2
:10486F006EE0900027F0121F0390006DE0FF121F03
:10487F000390006EE0FF121F0330280FC228900034
:10488F00337405F090000074F0F022900046E0FFC2
:10489F00121F3290003C740AF0900000E004F022E6
:10474D0090000DE0540F75F00AA4FFA3E0540F2F55
:10475D00F54F900010E0540F75F00AA4FF90000F74
:10476D00E0540F75F064A42FFF900011E0540F2F4B
:10477D00F550E54FC394014015E54FD39414500EF9
:10478D00E550C394014007E550D394FA400A1263F3
:10479D00BA90000074FAF02212661A900075EEF0CD
:1047AD00A3EFF0900075E475F001124213AFF0FE27
:1047BD00AD4F1249EC900010E0540F75F00AA4FFB4
:1047CD0090000FE0540F75F064A42FFF900011E0DE
:1047DD00540F2FF54F900075E0FEA3E0FFAD4F1283
:1047ED0049EC7BFF7A0E793A1263C090000074FE9B
:0247FD00F022A8
:103D0F007F0D12425BEF701A900010E0B43010A3D9
:103D1F00E0B4300BA3E0B43006A3E06430600302DC
:103D2F003DF9900014E0FF64306004EFB4350E905D
:103D3F000015E0540FD394054003023DF990001491
:103D4F00E0FF64316004EFB43611900019E0B42045
:103D5F0007900018E0B42003023DF9900014E0FF33
:103D6F0064326004EFB43710900018E0B42007906D
:103D7F000017E0B420028072900014E0FF643360FB
:103D8F0004EFB43809900015E0B42002805C900075
:103D9F0014E0FF64346005EF64397058900015E04B
:103DAF00540F75F00AA4FFA3E0540F2FF54F9000A6
:103DBF0018E0540F75F00AA4FF900017E0540F7528
:103DCF00F064A42FFF900019E0540F2FF550E54F2A
:103DDF00C394014015E54FD39414500EE550C3948E
:103DEF00014007E550D394FA400A1263BA900000DD
:103DFF0074FAF02212661A900075EEF0A3EFF090AD
:103E0F00003C740AF0E4F54F900041E0FFE54FC32A
:103E1F009F5027900075E475F001124213AFF0FE2A
:103E2F0090003CE0FD04F074032DF582E43400F5BE
:103E3F0083E0FD1249EC054F80CE7BFF7A0E793A75
:0A3E4F001263C090000074FEF02220
:104E1600900043E0FF700330285B121F3212661ABF
:104E2600900075EEF0A3EFF0E4F54F900041E0FF3F
:104E3600E54FC39F502C900075E475F001124213A4
:104E4600AFF0FE124A2D8F507423254FF582E434BD
:104E560000F583E550F07E00124A2D121F03054F20
:104E660080C9302810C228E54F04900033F0900026
:104E76000074F0F022900046E0FF121F3290003CD2
:0C4E8600740AF0D226900000E004F02234
:10536F00302365900001E0FF900034F0C223BF2A84
:10537F00079000007403F022900034E0FFB423087C
:10538F00900000E004F0803DEF547FFF121F039068
:10539F000034E0547FFF90003CE0FE04F074032ED5
:1053AF00F582E43400F583EFF0900041E02409FF2B
:1053BF00E433FE90003CE0D39FEE6480F874809855
:0953CF004006900000E004F02209
:1059DA0030234B900001E0FF900034F0C223BF2A2D
:1059EA00079000007403F022900034E0FFB4230B08
:1059FA00900000E004F0E004F080101267DE500F1F
:105A0A00900034E090003EF0900000E004F0227B29
:0F5A1A00FF7A0E791A1263C090000074FAF0221E
:10494F002023030249EB900001E0FF900034F0C2F6
:10495F0023BF2A079000007403F022900034E0FF79
:10496F00B4230A900000E004F0E004F0221267DEA6
:10497F00505B90003EE0540F75F00AA4FF90003496
:10498F00E0540F2FF0E0900C8693FF900034F0125C
:10499F001F03900034E0FF90003CE0FE04F074032E
:1049AF002EF582E43400F583EFF0900041E0240906
:1049BF00FFE433FE90003CE0D39FEE6480F87480F8
:1049CF0098900000E0400304F02214F0227BFF7A5D
:0D49DF000E791A1263C090000074FAF022E5
:106580003020099000DCE0F54D12669B302203E4D8
:10659000F54D30210B301E05754D0A8003754D28D1
:0765A000900000E004F0226E
:10530500E54D7065124349900040E0124235533532
:1053150064533A6E533A78533A82533A8C533F96D4
:105325005344A05349AA534EB45353BE0000535699
:105335001266E6801C12641C801712699180121295
:105345006992800D1269938008126994800312692D
:105355009530200F9000DEE09000A1F0900000E075
:0A53650004F0229000007401F02211
:1067CE009000A1E070091266B59000007401F022ED
:1056840030200D9000DCE0F54D12669BE54D70FC7A
:10569400302107754D05E54D70FCE4F54F30210CC4
:1056A40012682A12255612689C12255630200C12B4
:1056B400683512255612689C122556054FE54FC3CE
:1056C400940540D930200E9000DEE09000A1F090C7
:0C56D40000A1E070FA9000007401F022C8
:01698D0022E7
:01698E0022E6
:01698F0022E5
:104D1C0030210A201E079000007401F02230200D73
:104D2C009000DCE0F54D12669BE54D70FC302107E0
:104D3C00754D05E54D70FC30201B9000BFE0F52A49
:104D4C00126835E4F54F122556054FE54FC3940A0A
:104D5C0040F412689C30211B9000C0E0F52A1268C8
:104D6C002AE4F54F122556054FE54FC3940A40F43B
:104D7C0012689C30200E9000DEE09000A1F09000B4
:0D4D8C00A1E070FA121F6AE4900000F0220E
:0169900022E4
:105F380030133E20233B9000A47464F0E542547F64
:105F4800FF900A7D93900001F030260EE54230E77D
:105F580009EF900A8D93900001F0D223C2139000AC
:105F680001E0B42307900002E004F022E49000026C
:025F7800F02215
:105F7A0030113E20233B9000A47464F0E540547F26
:105F8A00FF900A7D93900001F030260EE54030E73D
:105F9A0009EF900A8D93900001F0D223C21190006C
:105FAA0001E0B42307900002E004F022E49000022A
:025FBA00F022D3
:10291300202403022AC5302303022AC5900002E0C3
:10292300F552E4F09000A47464F01269848F51D2DC
:1029330023E551B430079000017430F022E551B41F
:1029430031079000017431F022E551B43207900051
:10295300017432F022E551B433079000017433F06F
:1029630022E551B434079000017434F022E551B4E8
:1029730035079000017435F022E551B43607900015
:10298300017436F022E551B437079000017437F033
:1029930022E551B438079000017438F022E551B4B0
:1029A30039079000017439F022E551B423109000E7
:1029B300017423F0AF520552900002EFF022E5516B
:1029C300B42A07900001742AF022E551B44107901C
:1029D30000017441F022E551B442079000017442B2
:1029E300F022E551B443079000017443F022E5510E
:1029F300B464079000017444F022202603C223220A
:102A0300E551B461079000017461F022E551B462AD
:102A1300079000017462F022E551B463079000014E
:102A23007463F022E551B464079000017464F022EA
:102A3300E551B465079000017465F022E551B46671
:102A4300079000017466F022E551B4670790000116
:102A53007467F022E551B468079000017468F022AE
:102A6300E551B469079000017469F022E551B46A35
:102A730007900001746AF022E551B46B07900001DE
:102A8300746BF022E551B46C07900001746CF02272
:102A9300E551B46D07900001746DF022E551B46EF9
:102AA30007900001746EF022E551B46F07900001A6
:102AB300746FF022E551B470079000017470F02236
:032AC300C2232209
:0B67FA007F209000037420F0A3DFFC60
:016805002270
:0F67DE00EFC394304007EFD39439500122C32208
:104F800090000CE0FD6420602E90000BE0540F7543
:104F9000F00AA4FBAAF090000AE0540F75F064A494
:104FA0002BFFE5F03AFEED540F7C002FFFEC3E9016
:104FB0000071F0A3EF803190000BE0FD64209000C1
:104FC0000A601AE0540F75F00AA4FFED540F7C003C
:104FD0002FFEEC35F0900071F0A3CE800BE0540F63
:104FE000FF900071E4F0A3EFF0E024FFF090007177
:054FF000E034FFF02297
:10544000900009E0FD6420602B900008E0540F7587
:10545000F00AA4FBAAF0900007E0540F75F064A4D2
:105460002BFFE5F03AFEED540F7C002FFFEC3E9051
:105470000073802E900008E0FD6420900007601A01
:10548000E0540F75F00AA4FFED540F7C002FFEECE2
:1054900035F0900073F0A3CEF022E0540FFF90009F
:0754A00073E4F0A3EFF0221A
:10663D00900005E0540F75F00AA4FFA3E0540F2F4E
:10664D00900035F0D394004006E09415500122C31C
:01665D00221A
:10562700E4FFEF75F003A4249DF582E4340AF583C3
:10563700E493FE900004E0FDEE6D703BEF75F00320
:10564700A4249EF582E4340AF583E493FE900005D2
:10565700E0FDEEB50521EF75F003A4249FF582E484
:10566700340AF583E493FE900006E0FDEEB50507E6
:0C567700900036EFF0D3220FBF33A7C322
:015683002204
:10556900E4FF75F003EFA42436F582E5F0340BF57A
:1055790083E493FE900004E0FDEE6D703D75F00349
:10558900EFA42437F582E5F0340BF583E493FE901C
:105599000005E0FDEEB5052275F003EFA42438F50A
:1055A90082E5F0340BF583E493FE900006E0FDEE0E
:0F55B900B50507900037EFF0D3220FBF70A4C3E2
:0155C80022C0
:10425B0074032FF582E43400F583E0FD643170695B
:10426B00FE74042FF582E43400F583E0FCEE75F068
:10427B0003A4249DF582E4340AF583E4936C704225
:10428B0074052FF582E43400F583E0FCEE75F00342
:10429B00A4249EF582E4340AF583E493B5042374D5
:1042AB00062FF582E43400F583E0FCEE75F003A4F1
:1042BB00249FF582E4340AF583E493B50404EE04F9
:1042CB00FF220EBE339B7F0022ED6432706DFE74B5
:1042DB00042FF582E43400F583E0FD75F003EEA4C2
:1042EB002436F582E5F0340BF583E4936D70457459
:1042FB00052FF582E43400F583E0FD75F003EEA4A1
:10430B002437F582E5F0340BF583E493B50525747A
:10431B00062FF582E43400F583E0FD75F003EEA47F
:10432B002438F582E5F0340BF583E493B50505EEFF
:0D433B002434FF220EBE70977F00227F0009
:014348002252
:104B1A00EFC3943390006C50397431F0EF75F003A1
:104B2A00A4249DF582E4340AF583E49390006DF0A1
:104B3A00EF75F003A4249EF582E4340AF583E49326
:104B4A0090006EF0EF75F003A4249FF582E4340A16
:104B5A00803A7432F075F003EFA4249DF582E5F0F3
:104B6A00340AF583E49390006DF075F003EFA42402
:104B7A009EF582E5F0340AF583E49390006EF075B1
:104B8A00F003EFA4249FF582E5F0340AF583E49359
:054B9A0090006FF02205
:1066FD00900005E0540F75F00AA4FFA3E0540F2F8E
:05670D00900038F022AD
:10671200900005E0540F75F00AA4FFA3E0540F2F78
:05672200900039F02297
:10672700900005E0540F75F00AA4FFA3E0540F2F63
:0567370090003AF02281
:10661A0090004BE0FF90004AE08FF0A4FF90004901
:10662A00E07C002FFFEC35F0FE900042E02FFFECFB
:03663A003EFE22FF
:10673C00900044E075F010A4244DF9740235F0FA81
:05674C007BFF0263F178
:036984007F03226C
:1066E600302008900023E0FF126812302108900045
:0766F60023E0FF12680622F9
:10641C00E4F55E900033E0FFE55EC39F50217423EA
:10642C00255EF582E43400F583E0F55F302004FF4F
:0F643C00126812302105AF5F126806055E80D42A
:01644B00222E
:0169910022E3
:0169920022E2
:0169930022E1
:0169940022E0
:0169950022DF
:0C6806001268401225561268A3022556A5
:0C68120012684B1225561268A30225568E
:10434900E4F55EF55FF560900072E02401FF9000EE
:1043590071E03400FEC3EF940AEE94005005A3E027
:1043690004F560D3EF9463EE9400404C900072E042
:104379002401FB900071E03400FA7C007D64AF03F6
:10438900FE1241BE8F5EEF75F064A4FFC3EB9FFF81
:10439900EA95F0FE7C007D0A1241BE8F5FA3E0041E
:1043A900FFE55E75F064A4FEC3EF9EFFE55F75F05F
:1043B9000AA4FEC3EF9EF560900072E02401FF900D
:1043C9000071E03400FED3EF9409EE940040197CAB
:1043D900007D0A1241BE8F5FA3E004FFE55F75F01F
:1043E9000AA4FEC3EF9EF5607430255EF55E743055
:1043F900255FF55F74302560F560302014AF5E12DB
:104409006812AF5F126812AF601268127F2A1268D1
:1044190012302114AF5E126806AF5F126806AF60F2
:084429001268067F2A126806E2
:014431002268
:0663BA007BFF7A0D798AD9
:0663C0008B5F8A60896119
:1063C6007F01121F32E4F562AB5FAA60A9618562A4
:1063D6008275830012417FFF121F030562E562C3C7
:0463E600941040E4EB
:0163EA002290
:0663EB007BFF7A0D79DA58
:0663F1008B608A618962E5
:1063F7007F11121F32E4F563AB60AA61A96285635E
:106407008275830012417FFF121F030563E563C393
:04641700941040E4B9
:01641B00225E
:10603A007BFF7A0E794A1263F1126167E4F55EF525
:10604A005FE55F900A3C93FDAF5FAE5E1249ECE5F7
:10605A005F900A3C93FDAF5FAE5E125C80055FE520
:0E606A005F7002055EC3943AE55E940040D379
:016078002205
:0169960022DE
:0169970022DD
:0169980022DC
:0169990022DB
:01699A0022DA
:01699B0022D9
:01699C0022D8
:1065A7007BFF7A0E79CA1263C012603A126996129B
:1065B700699712699812699912699A12699B126907
:0765C7009C121F4C021F5B38
:10644C00755E01755F007560B3E4F561AF617E0048
:10645C00124A2DAB5E0560E560AA5F7002055F1401
:0E646C00F9EF1241AC0561E561C3943A40DEE0
:01647A0022FF
:10652F00126167E4F55EF55FAF5FAE5E124A2DADA7
:10653F0007AF5FAE5E125C80055FE55F7002055EC0
:09654F00C3943AE55E940040DFBC
:016558002220
:1065CE00E4F564F565AF65AE641264A9AD07AF6519
:1065DE00AE641249EC0565E56570020564C3943A34
:0665EE00E564940040DFAB
:0165F4002284
:1061DA00755E01755F007560B3E4F561F562AF62E3
:1061EA00AE611264A9AB5E0560E560AA5F70020544
:1061FA005F14F9EF1241AC0562E56270020561C3F2
:08620A00943AE561940040D6CE
:016212002269
:10621300755E01755F007560B3E4F561F562AB5EB1
:106223000560E560AA5F7002055F14F9124166FD1F
:10623300AF62AE611249EC0562E56270020561C3AB
:08624300943AE561940040D695
:01624B002230
:1049EC00C2B0758400D2C2C2C6D2C6C2C4D2C5C2BD
:1049FC00C330C3FD74A0F5C2C2C5C2C330C3FD8EA3
:104A0C00C2C2C330C3FD8FC2C2C330C3FD8DC2C28C
:104A1C00C330C3FDD2C4C2C320C4FD12253ED2B0E4
:104A2C0022758400C2C3D2C530C3FD74A0F5C2C2C6
:104A3C00C5C2C330C3FD8EC2C2C330C3FD8FC2C258
:104A4C00C330C3FDC2C4D2C5C2C330C3FD74A1F50B
:104A5C00C2C2C5C2C330C3FDC2C2C2C330C3FD850E
:104A6C00C207D2C4C2C320C4FD22D2C2C2C6D2C69F
:084A7C00D2C4C2C320C4FD2214
:102E1700754700122E3250FB22754700122EBB5009
:102E2700FB22754700122E7250FB22758400E5477E
:102E370075F003A4902E3F73022ED7022EE6022FC1
:102E470004022EED022F10022F17022F1F022EE66B
:102E5700022F2D022EED022F3D022F46022ED70202
:102E67002EE6022F54022EED022F60758400E547EF
:102E770075F003A4902E7F73022ED7022EE6022F41
:102E870004022EED022F10022F17022ED7022EE674
:102E9700022F04022EED022F10022F17022F10020D
:102EA7002F17022F1F022EE6022F62022EED022F8E
:102EB7003D022F60758400E54775F003A4902EC886
:102EC70073022ED7022EE6022F54022EED022F6038
:102ED700C2FA122F72122F72759B000547C3223058
:102EE700F9020547C32230F912E59A20E7FB122FB2
:102EF70072D2FA122F72122F720547C322C2FA1228
:102F07002F72759B040547C322753A1E0547C322D6
:102F1700E53A70020547C322C2FA122F72122F93A5
:102F2700F59B0547C322C2FA122F72122FA244073C
:102F3700F59B0547C322122F84F53B0547C322752E
:102F4700840F30DE04E53B70020547C322C2FA1244
:102F57002F72759B080547C322D322C2FA122F721C
:092F6700122FA24405F59B054759
:102F7000C32200000000000000000000000000006C
:102F800000000022902F8BE54893225A5A5A5A5A31
:102F9000FAFAFA902F9AE548932200B45AE12D8765
:102FA0007ADB902FA9E54893220000000000008002
:012FB00080A0
:105EB1002A2A3132333435362A2A2A2A31323334E6
:105EC10035302A2A44313233343536373839302A9D
:105ED10023414243202056455253494F4E20322EF2
:105EE10031322020202020205349454D454E53205A
:045EF100202020202D
:104B9F00302920C229E542540F905EC59390008CB6
:104BAF00F0786876329000B4E060151262ED126111
:104BBF002C800D7868E67008900078F0900089F0EE
:104BCF00302A3EC22AE540540F905EC59390008B69
:104BDF00F0754A32125CC9301E06740044B3700976
:104BEF00201E099000B5E060031260F1301E0674BC
:104BFF000044B37003201E031262B8201E13026319
:104C0F0056E54A700C900079F0900088F09000ED16
:024C1F00F02281
:1062B800900079E0FF04F0EF905EB193FF90008BBF
:1062C800E0FEEF6E6011EEB42A089000797401F0D8
:1062D8008005E4900079F0900079E0B40A06E4F0D3
:0562E800D221D22B229F
:1062ED00900078E0FF04F0EF905EB193FF90008C8A
:1062FD00E0FEEF6E6011EEB42A089000787401F0A4
:10630D008005E4900078F0900078E0B40A06E4F09F
:05631D00D220D22B226A
:1060F100900088E0FF04F0747F2FF582E43400F50E
:1061010083E0FF90008BE0FEEF6E6011EEB4230898
:106111009000887401F08005E4900088F090008878
:0B612100E0B40906E4F0D221D21F22F6
:10612C00900089E0FF04F0747F2FF582E43400F5D1
:10613C0083E0FF90008CE0FEEF6E6011EEB423085C
:10614C009000897401F08005E4900089F09000893A
:0B615C00E0B40906E4F0D220D21F22BC
:1063560090007BE0FF04F0EF905EBB93FF90008B14
:10636600E0FEEF6E6011EEB42A0890007B7401F037
:106376008005E490007BF090007BE0B40A04E4F032
:03638600D22C22F4
:1064D70090007F7423F0A3F0E4FF74B72FF582E4F4
:1064E7003400F583E0FE74812FF582E43400F583F0
:0C64F700EEF00FBF06E49000877423F065
:016503002275
:10598A00121E60121F4C7F01121F327BFF7A5E7952
:10599A00E51263C07BFF7A5E79D51263F17539141B
:1059AA00E490007EF090007DF0FF744C2FF582E4C5
:1059BA003400F583E4F0745C2FF582E43400F58357
:1059CA00E4F00FBF10E4E53970FC121F4C021F5BB4
:10514B0090007EE0FFD3940F501FEF04FF121F322D
:10515B0090008BE0FF90007EE0FE04F0744C2EF587
:10516B0082E43400F583EF80437F01121F32E4F5B4
:10517B005E744D255EF582E43400F583E0FF744CDC
:10518B00255EF582E43400F583EFF0744C255EF573
:10519B0082E43400F583E0FF121F03055EE55EC376
:1051AB00940F40CD90008BE0FF90005BF0121F033B
:0151BB0022D1
:1050680090007DE0FFD3940F5020EF2411FF121F12
:105078003290008CE0FF90007DE0FE04F0745C2E1E
:10508800F582E43400F583EF80437F11121F32E488
:10509800F55E745D255EF582E43400F583E0FF7407
:1050A8005C255EF582E43400F583EFF0745C255EE0
:1050B800F582E43400F583E0FF121F03055EE55E28
:1050C800C3940F40CD90008CE0FF90006BF0121F4E
:0150D80003D4
:0150D90022B4
:105CC9009000EDE0FF700E90008BE0B42A07900081
:105CD900ED7401F022EFB4011390008BE0B42307B7
:105CE9009000ED7402F022E49000EDF09000EDE0F8
:105CF900B4021490008BE0B430089000EE7401F007
:085D09008000E49000EDF0229F
:10443200E53760021537E53A6002153A900093E0DD
:10444200600214F0900097E0600214F090009BE08C
:10445200600214F090009FE0600214F09000A2E06D
:10446200600214F09000AAE0600214F09000B2E042
:10447200600214F022E538600215389000A1E06075
:104482000214F0900092E0600214F0900096E06056
:104492000214F09000A7E0600214F022E5396002F5
:1044A2001539E53B6002153BE54C6002154CE54DC4
:1044B2006002154D7868E6600116E54A6002154A09
:1044C200E54B6002154B9000AFE0600214F09000E3
:1044D2009AE0600214F090009EE0600214F09000F6
:1044E200A8E0600214F09000EFE0600214F02222D3
:1044F2009000A4E0600214F0229000A3E060021495
:02450200F022A5
:1020AA00202046554E4354494F4E20313820202097
:1020BA0000202020454D455247454E4359202020B7
:1020CA002000202020205354414E444259202020F1
:1020DA002020524144494F204F524947494E4154CA
:1020EA00452054454C434F204F524947494E41548D
:1020FA00452020202046554E4354494F4E2031203A
:10210A00202020202046554E4354494F4E2032204D
:10211A00202020202046554E4354494F4E2033203C
:10212A00202020202046554E4354494F4E2034202B
:10213A00202020202046554E4354494F4E2035201A
:10214A00202020202046554E4354494F4E20362009
:10215A00202020202046554E4354494F4E203720F8
:10216A00202020202046554E4354494F4E203820E7
:10217A00202020202046554E4354494F4E203920D6
:10218A002020202052454345495645204D4F44457D
:10219A002020205452414E534D4954204D4F44451E
:1021AA002020202046554E4354494F4E203130209E
:1021BA002020202046554E4354494F4E203131208D
:1021CA002020202046554E4354494F4E203132207C
:1021DA002020202046554E4354494F4E203133206B
:1021EA002020202046554E4354494F4E203134205A
:1021FA002020202046554E4354494F4E2031352049
:10220A002020202046554E4354494F4E2031362037
:10221A002020202046554E4354494F4E2031372026
:10222A002020202046554E4354494F4E2031382015
:10223A002020202046554E4354494F4E2031392004
:10224A002020202046554E4354494F4E20323020FC
:10225A002020202046554E4354494F4E20323120EB
:10226A002020202046554E4354494F4E20323220DA
:10227A002020202046554E4354494F4E20323320C9
:10228A002020202046554E4354494F4E20323420B8
:10229A002020202046554E4354494F4E20323520A7
:1022AA002020202046554E4354494F4E2032362096
:1022BA002020202046554E4354494F4E2032372085
:1022CA0020203A0036AA340031552EAA2C0029556E
:0E22DA0026AB240021551EAB1C001955140024
:101B75009000E8E07003021E5F202D0F9000B0E09A
:101B850060099000AFE07003021E5B202D03021E6A
:101B95005FC22D9000B0E0FF701DE540B40B0C90C6
:101BA50000AF7414F09000B0E004F0E540640C6000
:101BB50003021E5F021DD5EF64016003021CC8E528
:101BC50040B40B03021D7BE540B40C0D9000AF74CF
:101BD50014F09000B07404F0229000DBE0C394038D
:101BE500502EE54094004028E54094085022E540F9
:101BF500149000ACF09000AE7401F09000ACE0756C
:101C0500F010A424FCF9742035F0FA7BFF1263C0B0
:101C15009000DBE0B4032FE540D394074028E5406E
:101C2500940A5022E540149000ACF09000AE740187
:101C3500F09000ACE075F010A424FCF9742035F0A8
:101C4500FA7BFF1263C09000DBE064047035E54069
:101C55006408702F7BFF7A21796C1263C07BFF7A51
:101C650021799C1263F19000EBE0B403031268AA9A
:101C75009000ECE0B403031268B612669B9000B1C5
:101C85007401F09000DBE064047034E54064097091
:101C95002E7BFF7A21797C1263C07BFF7A21798CB8
:101CA5001263F19000EBE0B403031268B09000EC0E
:101CB500E0B403031268BC1266B5E49000B1F0E429
:101CC500021E5B9000B0E064036003021D6EE540F8
:101CD500B40C129000AF7414F0E49000F4F090008E
:101CE500B07405F022E540B40B03021DE7E540B4EE
:101CF500092E9000ACE09000ADF09000AC7414F0AB
:101D0500E49000ABF09000AE04F07BFF7A2079AA56
:101D15001263C07BFF7A2079BB1263F1E4021E5B7C
:101D25009000DBE0C394035007E540C394084005E9
:101D3500E540B40A30E540B40A089000AC7409F0F7
:101D45008008E54024099000ACF09000AE7401F0E5
:101D55009000ACE075F010A4241CF9742135F0FA5C
:101D65007BFF1263C0E4021E5B9000B0E064047068
:101D75004FE540B40C079000AF7414F022E540B471
:101D85000B02805E9000DBE0C39403502FE5409486
:101D9500004029E540940A5023E54024149000AC06
:101DA500F09000AE7401F09000ACE075F010A42442
:101DB500ECF9742035F0FA7BFF1263C0E4021E5B78
:101DC5009000B0E064056003021E5FE540B40C0DB1
:101DD5009000AF7414F09000B07403F022E540B4A5
:101DE5000B0D9000AF7414F09000B07401F02290C8
:101DF50000DBE0C39403505DE540C3940B5056905F
:101E050000AF7414F0E5409000F4B40A12E0FF044A
:101E1500F074F02FF582E43400F583E4F08011E0EE
:101E2500FF04F074F02FF582E43400F583E540F00B
:101E35009000F4E0D3940340219000F0E094085022
:101E45000E9000F2E0C3940850051267518003120A
:0B1E5500667DE48001E49000B0F02204
:1017D5009000DBE064047003021B749000AEE070BF
:1017E50003021B7412694E9000ABE0FF703090004D
:1017F500ACE0FE64076011EEC39405400BEED39494
:1018050013400CEE941850079000AB7401F022EED3
:101815009000ABB408047408F0227404F022EFB40D
:1018250001030219599000ABE0640260030218E05D
:101835009000AAE06003021B749000ACE0FF600317
:10184500B4070C9022D0E493F516740193F517EFC5
:10185500B4010C9022D2E493F516740193F517EFB9
:10186500B4020C9022DCE493F516740193F517EF9E
:10187500B4030C9022DEE493F516740193F517EF8B
:10188500B4040C9022D8E493F516740193F517EF80
:10189500B4140C9022CEE493F516740193F517EF6A
:1018A500B4150C9022DAE493F516740193F517EF4D
:1018B500B4160C9022D4E493F516740193F517EF42
:1018C500B4170C9022D6E493F516740193F517908E
:1018D50000C4E0F528126954021A569000ABE06482
:1018E50003706A9000AAE06003021B749022CC93F7
:1018F500F516740193F5179000C5E0F528126954A3
:101905009000B17401F0126930E49000ABF09000E2
:10191500AEF09000ACE064146003021B749000AD5F
:10192500E09000ACF0126957121F4CE49000B1F042
:1019350090009CF0900099F09000DEE0FF9000D9B7
:10194500E02F9000A1F09000A5740AF0229000AB62
:10195500E0B404209022CCE493F516740193F517B6
:101965009000C6E0F52812695412694E9000AA74D9
:1019750078021B269000ABE0FF64056003021A5E47
:101985009000AAE06003021B749000ACE0FEB40571
:101995000C9022E0E493F516740193F517EEB40666
:1019A5000C9022E2E493F516740193F517EE6409A1
:1019B5006004EEB4180C9022E0E493F516740193DC
:1019C500F517EE640A6004EEB4190C9022E0E49376
:1019D500F516740193F517EE640B6004EEB41A0C5A
:1019E5009022E0E493F516740193F517EEB40C0C10
:1019F5009022E0E493F516740193F517EEB40D0CFF
:101A05009022E2E493F516740193F517EE640E60E7
:101A150004EEB41B0C9022E2E493F516740193F5E1
:101A250017EE640F6004EEB41C0C9022E2E493F50B
:101A350016740193F517EE64106004EEB41D0C9056
:101A450022E2E493F516740193F5179000C4E0F5CE
:101A5500289000AA7428021B26EF64066003021B67
:101A65002E9000AAE06003021B749000ACE0FF64B6
:101A7500056004EFB4060C9022D0E493F5167401CA
:101A850093F517EF64096004EFB40D0C9022D2E4CE
:101A950093F516740193F517EF640A6004EFB40E1D
:101AA5000C9022DCE493F516740193F517EF640BA3
:101AB5006004EFB40F0C9022DEE493F516740193E5
:101AC500F517EF640C6004EFB4100C9022D8E49382
:101AD500F516740193F517EF64186004EFB41B0C49
:101AE5009022DAE493F516740193F517EF64196003
:101AF50004EFB41C0C9022D4E493F516740193F50D
:101B050017EF641A6004EFB41D0C9022D6E493F528
:101B150016740193F5179000C4E0F5289000AA7497
:101B250028F09000ABE004F0229000ABE0FFB40792
:101B3500279000AAE070389022CC93F51674019393
:101B4500F5179000C5E0F5289000B17401F0E49018
:101B550000ABF09000AEF022EFB4081312695712F3
:101B65006951E49000ABF09000AEF09000B1F02226
:10251200000000000000000000000000000022C0D7
:1025220000C001790478B4D8FED9FAD001D00022D3
:10253200C0007814122521D8FBD00022C0E07537E4
:1025420005E53770FCD0E022C0E075370FE5377043
:10255200FCD0E022C0E0753764E53770FCD0E022A1
:10256200A42582F582E58335F0F58322B40A0022A0
:10257200C0E0C3997001D3D0E022B5060122500712
:10258200B5070122400122D322EF75F06484243082
:1025920090006CF0E5F0A375F00A842430F0A3E516
:1025A200F02430F022EF75F06484243090006CF057
:1025B200E5F0A375F00A842430F0A3E5F02430F0AE
:1025C20090006CE0B4300B7420F0A3E0B4300374DC
:1025D20020F02290000DE0540FFFA3E0B42002800F
:1025E20019540FCF75F00AA42FFFA3E0B420028084
:1025F20009540FCF75F00AA42FFF22C006C005C0F0
:082602000490000DE0540FFFED
:10260A00FEA3E0B42003C3802C540FFDCF75F00A5B
:10261A00A42FFFA3E0B42003C3801A540FFCEE7565
:10262A00F064A420D20EFEED75F00AA42E40052C0B
:10263A0040028001D3D004D005D0062275F064840C
:10264A00F6E5F00875F00A84F608A6F00822C0013B
:10265A007900E6B4FF028027F908E6B4FF03C380D5
:10266A0022E975F00AA426F908E6B4FF03C3801329
:10267A00E975F00AA420D207C3264003F98004D3DF
:10268A00D00122E9D00122E675F00AA408262278B0
:10269A0047EE12264675450075460078499026F29F
:1026AA007908EF134007A3A3A3A3A3801CC0E0C02B
:1026BA0000C001C37905E49336D4A2E4540FF6A30B
:1026CA0018D9F3D001D000D0E0D9D8E545600C750F
:1026DA004609754709754809754909854645854773
:1026EA004685484785494822060502000002010539
:1026FA0000000402000100080400020006090004A8
:10270A00000209010800040803060108060702037B
:1022E80020205455524E204F4E2053572020202056
:1022F8000020205455524E204F4646205357202048
:10230800200044313233343536373839302A2341C6
:10231800424302AB055508000AAB0D55100012AB3D
:10232800155518001AAB1D55200022AB255528005D
:102338002AAB2D55300032AA355520205445535428
:1023480020524F5554494E4520202020564552537F
:10235800494F4E20312E30202020205445535449D7
:102368004E4720454550524F4D2020205445535448
:10237800494E4720564F4943452020544553544918
:102388004E472044544D462031202054455354494B
:102398004E472044544D4620322020205445535463
:1023A800494E47205253323332202020544553544B
:1023B800494E472052533438352020202054455365
:1023C80054494E47205054542020205445535420FB
:1023D8004155582052454C415920205445535420CA
:1023E80043542052454C4159202020544553494ECE
:1023F800472052494E47494E472020202020202080
:102408002020202020202020202020544553542004
:102418004C494E452052414C415954455354204C47
:10242800494E452053454E53452B54455354204C53
:10243800494E452053454E53452D2020544553546D
:10244800204449475F494E202020205445535420BA
:10245800494E50555420564F4C54205445535420FF
:102468004C494E452052454C415954455354205AE5
:1024780045524F2043524F53532054455354494ECD
:102488004720535155454C43482020205445535428
:10249800494E472048504620202020544553542078
:1024A80054454C434F20564F5820205445535420F0
:1024B800524144494F20564F5820205445535420E8
:1024C800454D5F4F505450202020202020202020B0
:1024D80020202020202020202020202020202020F4
:1024E8002020202020202020202020544553542024
:1024F800434F4D504C4554454420202020544553CB
:0A25080054204641494C4544202070
:100EDA007BFF7A2379421263C07BFF7A237952120D
:100EEA0063F112686C7BFF7A2379621263C0121F66
:100EFA005B12686C7F007E00124A2D8F4F7DAA7F9D
:100F0A00007E001249EC7F007E00124A2DEF64AA8F
:100F1A00600C7BFF7A2579021263F11269877D558D
:100F2A007F007E001249EC7F007E00124A2DEF649A
:100F3A0055600C7BFF7A2579021263F1126987AD3D
:100F4A004F7F007E001249EC7BFF7A2479F212630C
:100F5A00C012686C7BFF7A2379721263C01268C868
:100F6A0012682A754700754801753914122E29E549
:100F7A003970FC122E2012690475470075480175F4
:100F8A003905E53970FCD202D20A122E17C202C202
:100F9A000A7BFF7A2479F21263C012686C7BFF7AAB
:100FAA002379821263C0121F5B12686C7F31126848
:100FBA004B753932E53970FC1268A33013FD12689B
:100FCA00A3E542547FFFEF90230A93FFEFB4310E5B
:100FDA007BFF7A2479F21263C012686C800C7BFF63
:100FEA007A2579021263F11269877BFF7A23799253
:100FFA001263C0121F5B12686C7F3112684012685C
:10100A00741268A33011FDE540547FFFEF90230A64
:10101A0093FFEFB4310E7BFF7A2479F21263C01288
:10102A00686C800C7BFF7A2579021263F11269875A
:10103A007BFF7A2379A21263C0121F5B12686C7558
:10104A008400759850C299C2987599433098FD7575
:10105A008400E5996443600C7BFF7A257902126368
:10106A00F11269877BFF7A2479F21263C012686CE5
:10107A007BFF7A2379B21263C0121F5B12686C126B
:10108A00690C758400759850C299C2987599433055
:10109A0099FD7BFF7A2479F21263C012686C7BFF98
:1010AA007A2379C21263C0121F5B12686C12669BA4
:1010BA00126874E53ED39432400C7BFF7A2579029C
:1010CA001263F11269871266B5126874E53EC39419
:1010DA00AA500C7BFF7A2579021263F11269877B89
:1010EA00FF7A2479F21263C012686C7BFF7A237943
:1010FA00D21263C0121F5B12686C1268AA1268745B
:10110A00E53DD3940A400C7BFF7A2579021263F1FC
:10111A001269871268B0126874E53DC394AA500C2C
:10112A007BFF7A2579021263F11269877BFF7A24A1
:10113A0079F21263C012686C7BFF7A2379E2126338
:10114A00C0121F5B12686C1268B612686C12686C67
:10115A001268BC7BFF7A2479F21263C012686C7B36
:10116A00FF7A2479121263C0121F5B12686C12682C
:10117A00C212686C12686C1268C812686C12686CC9
:10118A007BFF7A2479421263C0121F5B12686C30AB
:10119A00DC1D7BFF7A2279E81263F120DCFD121F45
:1011AA005B7BFF7A2479F21263C012686C801B7B26
:1011BA00FF7A2279F91263F130DCFD121F5B7BFFA3
:1011CA007A2479F21263C012686C7BFF7A2479C29E
:1011DA001263C0121F5B12686C1268EC501F7BFF0F
:1011EA007A2279E81263F11268EC40FB121F5B7BEA
:1011FA00FF7A2479F21263C012686C801D7BFF7A31
:10120A002279F91263F11268EC50FB121F5B7BFF23
:10121A007A2479F21263C012686C7BFF7A247952BD
:10122A001263C0121F5B12686CE53CC3940A400744
:10123A00E53CD39446400C7BFF7A2579021263F190
:10124A001269877BFF7A2479F21263C012686C7B79
:10125A00FF7A2479721263C0121F5B12686C1268DB
:10126A005612692740FB12692750FB12692740FB77
:10127A007BFF7A2479F21263C012686C12689C7B35
:10128A00FF7A2479821263C0121F5B12686C12689B
:10129A00CE400F12669B1266B51268CE50F58002D8
:1012AA0080F17BFF7A2479F21263C012686C7BFFAB
:1012BA007A2479B21263C0121F5B12686C126861D9
:1012CA001268D450FB800280F712689C7BFF7A2454
:1012DA0079F21263C012686C7BFF7A2479921263E6
:1012EA00C0121F5B12686C12685612687C90231C2D
:1012FA00E493F508740193F50912687C90231EE4BF
:10130A0093F508740193F50912687C902320E493FD
:10131A00F508740193F50912687C902322E493F589
:10132A0008740193F50912687C902324E493F50864
:10133A00740193F50912687C902326E493F50874E6
:10134A000193F50912687C902328E493F508740147
:10135A0093F50912687C90232AE493F508740193A3
:10136A00F50912687C90232CE493F508740193F52F
:10137A000912687C90232EE493F508740193F50909
:10138A0012687C902330E493F508740193F50912EE
:10139A00687C902332E493F508740193F509126886
:1013AA007C902334E493F508740193F50912687C60
:1013BA00902336E493F508740193F50912687C903A
:1013CA002338E493F508740193F50912687C902395
:1013DA003AE493F508740193F50912687C90233C6A
:1013EA00E493F508740193F50912687C90233EE4AE
:1013FA0093F508740193F50912687C902340E493ED
:10140A00F508740193F50912689C7BFF7A2479F236
:09141A001263C012686C0212F1A9
:0114230022A6
:08686C0075390AE53970FC22C0
:08687400753902E53970FC22C0
:08687C00753905E53970FC22B5
:0369870080FE226D
:08000300022AC6000000000003
:08000B00022AC70000000000FA
:08001300022BFA0000000000BE
:08001B003200000000000000AB
:09002300320000000000000000A2
:08002B00022ACA0000000000D7
:08003300320000000000000093
:0A003B003200000000000000000089
:0900430032000000000000000082
:08004B0032000000000000007B
:08005300320000000000000073
:08005B00022B2C000000000044
:08006300320000000000000063
:08006B00022B4B000000000015
:08007300022AD0000000000089
:08007B00022BFB000000000055
:08008300022B2900000000001F
:08008B0032000000000000003B
:10009300022C190000000000000000000000000016
:1000A3003275FF0775FFDE75FFAD75840F75E107C8
:1000B30075E20475E34475840F75A43575A5097558
:1000C300A6FF75A7FF759CFF759D00759E00759F24
:1000D300F075D8FF75E8FF75F80F75AD0F758401DE
:1000E30075893075888F75840275893075888F7529
:1000F300840F758A80758C67780874FF0000000090
:100103000000000000000000D5E0F1D8EDE58C30E0
:10011300E7FB759701758A0043890475840075B7F9
:100123001075840F438901758D01758F01758E02DA
:100133007480D5E0FD438902E58930E4FB759702BD
:1001430075840075D10775840075BB0175BA007598
:10015300BCF075C70075C60075C5FF75C4FF75E8AB
:100163008175840275BB0475BA0075BCF175C60050
:1001730075C4FF75E88875840075D484758401752A
:10018300D484758400C2F8759A47759D1A43F8099B
:1001930075870075840075B90075A90075910075A0
:1001A300985075840175981075840075C04075C3A7
:1001B3000075CFC9758400758E0075892075880513
:1001C300758400758A00758B6F758CF4758D6F431C
:1001D300885075840075C90075CA0075CB0075CC4D
:1001E3000075CD0075840175C91875CA8075CBFB80
:1001F30075CDFB75CC80D2CA75840275C91875CAD2
:10020300A675CBAF75CDAF75CCA6D2CA7584007574
:10021300A8AF75B80075E6A475E71775F60075F70E
:10022300019000007F007E20E4F0A3DFFCDEFA757E
:0202330027FFA3
:100235007528FF7529FF752AFF752BFF752CFF752E
:080245002DFFD2B6124A762209
:105C8000AC84A2AF922EABB1C2AF75840F53A1FE0C
:105C900075B121E4F58443B701F584438F01786C35
:105CA000768008F6EF26F618EE36F6E6FE08E6F5FC
:105CB000828E83EDF0E4F584538FFEF58453B7FEB6
:085CC0008BB18C84A22E92AF7F
:015CC80022B9
:1064A900AD84A2AF922EACB1C2AF75B12175668031
:1064B900756700EF2567F567EE3566F566856782CE
:0D64C900F583E493FF8CB18D84A22E92AF79
:0164D60022A3
:10616700AF84A2AF922EAEB1C2AF786C76800876BC
:106177000075B121E4F58443B701F584758F0318E1
:10618700E6FC08E6F5828C83E4F0F58FF58453B7D7
:09619700FE8EB18F84A22E92AF9E
:0161A00022DC
:1048AF0008D0094E09D40A600AF40B910C360CE5B6
:1048BF000D9D0E600F2D100610EB11DD12DC13EAAB
:1048CF0015071633177118C01D2107B107E8082007
:1048DF000859196E1A211ADA1B971C5A0894090ED7
:1048EF0009900A190AA90B410BE30C8C0D3F0DFD22
:1048FF000EC50F9810771162125B13621477159B18
:10490F0016D018161DEF1EC21F9B2079215F224A59
:10491F00233B2434253326392747285C29792A9DC0
:10492F002BC92CFE2E3B2F8230D032293379350AFA
:10493F00367F3641397B3AFE3C943E41400741D1A8
:0F679C0075F002124229E493F508740193F50990
:0367AB00D21522E2
:03698A00C2152211
:0868840075391EE53970FC2294
:08688C00753950E53970FC225A
:08689400753864E53870FC2240
:104D990012698A9000F0E0540F75F014A424AFF55D
:104DA90082E43448F583C083C0829000F1E0540F57
:104DB900D082D08312679C9000F2E0540FFF9000DC
:104DC900F0E0540FB507159000F3E0540FFF900081
:104DD900F1E0540FB5070512688C802D1268941202
:104DE900698A9000F2E0540F75F014A424AFF5829B
:104DF900E43448F583C083C0829000F3E0540FD0B7
:0D4E090082D08312679C12688412698A228D
:106751009000BFE0F52A126942126972124D991236
:056761006945026975A5
:10667D009000B6E060031269519000BFE0F52A1258
:0E668D00697212685612686C12697502694EC5
:0300000002681E75
:0C681E00787FE4F6D8FD75816D0245041A
:10416600BB010689828A83E0225002E722BBFE0257
:09417600E32289828A83E493228A
:10417F00BB010CE58229F582E5833AF583E02250F5
:10418F0006E92582F8E622BBFE06E92582F8E2223F
:0D419F00E58229F582E5833AF583E4932259
:1041AC00BB010689828A83F0225002F722BBFE01F2
:0241BC00F322EC
:1041BE00BC000BBE0029EF8DF084FFADF022E4CCE5
:1041CE00F875F008EF2FFFEE33FEEC33FCEE9DECAE
:1041DE00984005FCEE9DFE0FD5F0E9E4CEFD22EDF4
:1041EE00F8F5F0EE8420D21CFEADF075F008EF2F3E
:1041FE00FFED33FD4007985006D5F0F222C398FD2F
:05420E000FD5F0EA22CB
:10421300A3F8E0C5F025F0F0E5821582700215835E
:06422300E0C838F0E822BB
:0C422900A42582F582E5F03583F58322A0
:10423500D083D082F8E4937012740193700DA3A318
:1042450093F8740193F5828883E47374029368602C
:06425500EFA3A3A380DF2C
:00000001FF
